:060000000C9401120C94A7
:1000060000000C9400000C9400000C9400000C946A
:1000160000000C9400000C948E270C9400000C94A5
:1000260000000C9451150C9400000C9400000C94E4
:1000360000000C9400000C9400000C94F1140C9435
:1000460000000C9474260C9400000C948D260C94DD
:1000560000000C9400000C9400000C9400000C941A
:1000660000000C9400000C9400000C9400000C940A
:1000760000000C94B2260C9400000C944D270C94AE
:1000860000000C940000100000010204081020403B
:100096008000000040008000C00000014001050013
:1000A600C11100000300D90B00000300C1110300B9
:1000B600170E0300D90B00000500E00800000A0037
:1000C600C1110A00170E0A00D90B0A00C1110A0055
:1000D600170E2800D90B00000000000000000000E9
:1000E600000000000000000000000000000000000A
:1000F6000000000000000000070018C0202020209B
:100106004D904D90401040104890471020202020E0
:1001160018C007000000000007001FC03FE03FE0D6
:10012600727072707FF07FF0777078F03FE03FE09A
:100136001FC007000000000007800F100E300C7073
:1001460008F001F003F007F007F003F001F008F003
:100156000C700E300F1007001E008F00C700E30062
:10016600F100F800FC00FE00FE00FC00F800F100C3
:10017600E300C7008F001E007E0081008100810021
:1001860081008100FF00810081008100FF00810065
:100196008100810081007E00000000000200020054
:1001A60007000F801FC03FE03FE03FE01AC0070096
:1001B6000F800000000000000000000000000000AA
:1001C6000000000006000F000F00060000000000FF
:1001D6000000000000000000FFF0FFF0FFF0FFF05D
:1001E600FFF0FFF0F9F0F0F0F0F0F9F0FFF0FFF0BB
:1001F600FFF0FFF0FFF0FFF000000000000000003D
:10020600060009001080108010801080090006008A
:100216000000000000000000FFF0FFF0FFF0FFF01C
:10022600F9F0F6F0EF70EF70EF70EF70F6F0F9F0AE
:10023600FFF0FFF0FFF0FFF000000000000001E01B
:1002460000601EA0332061806180618033001E0043
:1002560000000000000000000000000007800CC045
:100266001860186018600CC00780030003000FC0F8
:10027600030003000000000002000300038003C027
:1002860002C002C00280020002000E001E001E0014
:100296000C000000000000000C000E000B0009809E
:1002A6000CC00E400B4009C038C07840784031C0C1
:1002B60003C003C0018000000000020002002720E6
:1002C6001FC018C030607070306018C01FC0272073
:1002D60002000200000000000000000010001800EC
:1002E6001C001E001F001F801F001E001C0018009F
:1002F60010000000000000000000000000800180E7
:10030600038007800F801F800F8007800380018095
:1003160000800000000000000000020007000F80BF
:100326001FC0020002000200020002001FC00F8070
:1003360007000200000000000000198019801980E3
:100346001980198019801980198019801980000078
:10035600198019800000000000001FE036C066C04A
:1003660066C066C036C01EC006C006C006C006C04F
:1003760006C006C00000000000001F8030C030002C
:1003860030001F8030C030C01F8000C000C030C0A9
:100396001F800000000000000000000000000000B8
:1003A60000000000000000000000000000001FE048
:1003B6001FE01FE000000000020007000F801FC0C2
:1003C6000200020002000200020002001FC00F80AD
:1003D600070002001FC000000000020007000F8097
:1003E6001FC002000200020002000200020002001A
:1003F60002000200000000000000020002000200ED
:100406000200020002000200020002001FC00F806C
:1004160007000200000000000000000000000000CD
:100426000100018001C03FE001C001800100000021
:1004360000000000000000000000000000000000B6
:1004460004000C001C003FE01C000C00040000002F
:100456000000000000000000000000000000000096
:100466000000000000000000400040004000400086
:1004760040007FE0000000000000000000000000D7
:10048600088018C038E07FF038E018C00880000007
:100496000000000000000000000000000000000056
:1004A6000000020007000F801FC03FE07FF0000041
:1004B6000000000000000000000000000000000036
:1004C60000007FF03FE01FC00F8007000200000021
:1004D6000000000000000000000000000000000016
:1004E6000000000000000000000000000000000006
:1004F6000000000000000000060006000F000F00CC
:100506000F000F000F0006000600060000000000A6
:100516000600060000000000000000001980198097
:100526001980198000000000000000000000000093
:100536000000000000000000000006600660066083
:100546003FF00CC00CC0198019807FC03300330007
:100556003300000000000000060006001F803FC0B8
:10056600360036003F801FC006C006C03FC01F8051
:1005760006000600000000000000000000103830F1
:10058600387038E001C0038007000E001C0038E018
:1005960070E060E000000000000007000D80198098
:1005A60019801B000E001E003E00336033C03180F0
:1005B6003BC01E60000000000E000E000E0006008C
:1005C60006000C0000000000000000000000000013
:1005D6000000000000000000038006000E000C0072
:1005E6001C001C001C001C001C001C000C000E0043
:1005F60006000380000000001C0006000700030040
:1006060003800380038003800380038003000700C8
:1006160006001C000000000000000000000036C0BC
:1006260036C01F800F003FC00F001F8036C036C087
:1006360000000000000000000000000000000000B4
:100646000600060006003FC03FC006000600060082
:100656000000000000000000000000000000000094
:1006660000000000000000000000000000000E0076
:100676000E000E0006000C00000000000000000046
:100686000000000000003FC03FC000000000000066
:100696000000000000000000000000000000000054
:1006A60000000000000000000000000000000E0036
:1006B6000E000E0000000000000000100030007068
:1006C60000E001C0038007000E001C003800700027
:1006D60060000000000000000F803FE030606070A6
:1006E60060F061B0633066306C3078307030306006
:1006F6003FE00F8000000000030007001F001F00FE
:1007060003000300030003000300030003000300CB
:100716001FE01FE0000000001FC03FE07070603067
:10072600607000E001C0038007000E001C00380066
:100736007FF07FF0000000001FC03FE07070603067
:10074600003000700FE00FC0006000306030707045
:100756003FE01FC00000000001C003C007C00EC07C
:100766001CC038C070C060C07FF07FF000C000C001
:1007760000C000C0000000007FF07FF06000600055
:1007860060007FC03FE00070003000306030707065
:100796003FE01FC00000000003C007C00E001C00A1
:1007A600380030007FC07FE070706030603070705D
:1007B6003FE01FC0000000007FF07FF00060006097
:1007C60000C000C00180018003000300060006008F
:1007D6000C000C00000000000F801FC038E03060E5
:1007E600306038E01FC03FE070706030603070707D
:1007F6003FE01FC0000000001FC03FE07070603087
:10080600603070703FF01FF0006000E001C00380B0
:100816001F001E0000000000000000000000000095
:100826000E000E000E000000000000000E000E007C
:100836000E000000000000000000000000000000A4
:100846000E000E000E000000000000000E000E005C
:100856000E00060006000C0000C001C00380070061
:100866000E001C00380038001C000E000700038034
:1008760001C000C0000000000000000000000000F1
:1008860000003FE03FE0000000003FE03FE00000E6
:100896000000000000000000300038001C000E00C0
:1008A6000700038001C001C0038007000E001C0082
:1008B60038003000000000001F803FC070E060601C
:1008C60060E001C003800700060006000600000085
:1008D60006000600000000001FC03FE0306067B061
:1008E6006FB06DB06DB06DB06DB06FE067C0700089
:1008F6003FC00FC000000000060006000F000F00FA
:100906000F0019801980198030C03FC03FC0606059
:1009160060606060000000007F007F8061C060C092
:1009260060C061C07F807FC060E06060606060E042
:100936007FC07F80000000000F801FC038E030605D
:10094600600060006000600060006000306038E0B9
:100956001FC00F80000000007F007F8061C060C064
:1009660060606060606060606060606060C061C0C0
:100976007F807F00000000007FE07FE06000600075
:10098600600060007F807F80600060006000600023
:100996007FE07FE0000000007FE07FE06000600015
:1009A600600060007F807F80600060006000600003
:1009B60060006000000000000FC01FE038603000DB
:1009C6006000600063E063E0606060603060386033
:1009D6001FE00FE000000000606060606060606023
:1009E600606060607FE07FE06060606060606060C3
:1009F60060606060000000001F801F800600060027
:100A060006000600060006000600060006000600B0
:100A16001F801F8000000000006000600060006012
:100A2600006000600060006000606060606070C030
:100A36003FC01F8000000000606060E061C063800E
:100A460067006E007C007C006E006700638061C0FA
:100A560060E0606000000000600060006000600010
:100A66006000600060006000600060006000600080
:100A76007FE07FE000000000606070E070E079E0F9
:100A860079E06F606F60666066606060606060609D
:100A96006060606000000000606070607060786098
:100AA6006C606C60666066606360636061E060E015
:100AB60060E06060000000000F001F8039C030C099
:100AC60060606060606060606060606030C039C0B7
:100AD6001F800F00000000007F807FC060E0606024
:100AE6006060606060E07FC07F80600060006000E2
:100AF60060006000000000000F001F8039C030C099
:100B060060606060606060606060636033C039C070
:100B16001FE00F60000000007F807FC060E0606023
:100B26006060606060E07FC07F806700638061C056
:100B360060E06060000000001F803FC070E0606001
:100B4600600070003F801FC000E00060606070E0E1
:100B56003FC01F80000000003FC03FC006000600E7
:100B6600060006000600060006000600060006004F
:100B76000600060000000000606060606060606063
:100B8600606060606060606060606060606030C02F
:100B96003FC01F800000000060606060606030C081
:100BA60030C030C01980198019800F000F000F0067
:100BB6000600060000000000606060606060606023
:100BC600606060606060666066606F6079E070E0DB
:100BD60070E06060000000006060606030C030C09F
:100BE60019800F00060006000F00198030C030C0C3
:100BF60060606060000000006060606030C030C00F
:100C0600198019800F000F00060006000600060076
:100C160006000600000000007FE07FE000C000C084
:100C260001800300060006000C00180030003000AA
:100C36007FE07FE000000000666066600F000F0046
:100C46000F0019801980198030C03FC03FC0606016
:100C560060606060000000006F605FA039C030C057
:100C660060606060606060606060606030C039C015
:100C76001F800F0000000000606060600000606080
:100C8600606060606060606060606060606030C02E
:100C96003FC01F80000000001F801F801800180042
:100CA600180018001800180018001800180018007E
:100CB6001F801F80000000000000000000000000F0
:100CC600000000000000000000000000000000001E
:100CD600000000007FF07FF000000700070007001B
:100CE60006000600030000000000000000000000EF
:100CF60000000000000000000000000000000000EE
:100D060000001FC03FE000601FE03FE060606060E1
:100D16007FE03FE0000000006000600060006000CF
:100D260060006F807FC070E060606060606060E05F
:100D36007FC07F800000000000000000000000006F
:100D460000001F803FC0706060006000600070603F
:100D56003FC01F800000000000600060006000606F
:100D660000601F603FE071E060606060606070601E
:100D76003FE01FE00000000000000000000000004F
:100D860000001F803FC070607FE07FC06000700081
:100D96003FC01F800000000007800F801C00180065
:100DA600180018007F007F001800180018001800AF
:100DB60018001800000000000000000000000000FD
:100DC60000001FE03FE07060606070E03FE01F6081
:100DD600006000E03FC03F8060006000600060008F
:100DE60060006F007F8071C060C060C060C060C07E
:100DF60060C060C0000000000000000006000600A1
:100E060000000E000E0006000600060006000600A2
:100E16001F801F800000000000000000018001808C
:100E26000000038003800180018001800180018031
:100E3600018019801F800F00300030003000300024
:100E460030003180338037003E003E00370033806B
:100E560031C030C0000000000E000E000600060083
:100E6600060006000600060006000600060006004C
:100E76001F801F800000000000000000000000002E
:100E8600000059807FC07FE06660666066606660CD
:100E960066606660000000000000000000000000C0
:100EA60000003F803FC030E030603060306030602E
:100EB600306030600000000000000000000000000C
:100EC60000001F803FC070E060606060606070E09E
:100ED6003FC01F800000000000000000000000006E
:100EE60000007F807FC060E06060606070E07FC06F
:100EF6006F806000600060000000000000000000DD
:100F060000001FE03FE070606060606070E03FE0FE
:100F16001F6000600060006000000000000000002C
:100F2600000037C03FE0386030003000300030004D
:100F3600300030000000000000000000000000004B
:100F460000003F007F8060007F003F8001800180BD
:100F56007F803F0000000000000018001800180005
:100F660018007F007F0018001800180018001800ED
:100F76001F800F800000000000000000000000003D
:100F8600000060606060606060606060606070E08B
:100F96003FE01F60000000000000000000000000AD
:100FA60000006060606030C030C0198019800F009A
:100FB6000F00060000000000000000000000000016
:100FC6000000666066606660666066606F603FC06F
:100FD60039C0108000000000000000000000000082
:100FE600000060C071C03B801F000E001F003B80E8
:100FF60071C060C00000000000000000000000009A
:10100600000030C030C0198019800F000F000600A4
:1010160006000C000C001800000000000000000094
:1010260000007FC07F80030006000C00180030001F
:101036007FC07FC00000000000000000606000006C
:1010460000001FC03FE000601FE03FE0606060609E
:101056007FE03FE00000000000000000606000004C
:1010660000001F803FC070E060606060606070E0FC
:101076003FC01F800000000000000000606000000C
:10108600000060606060606060606060606070E08A
:101096003FE01F600000000000003F007F8060C04E
:1010A60060C061C0678067C060E06060606060E0EB
:1010B60067C067800000000000000000000000001C
:1010C60006000F00198030C0606060607FE07FE03E
:1010D60000000000000000000F801FC038E03060F4
:1010E60060606000600060006000306038E01FC033
:1010F6000F8006001E001E000000000019801980E7
:10110600000060606060606060606060606070E009
:101116003FE01F60000000000000018003000600A1
:1011260000001F803FC070607FE07FE060007000BD
:101136003FC01F8000000000000006000F0019805D
:1011460000001FC03FE000601FE03FE0606060609D
:101156007FE03FE0000000000000000019801980D9
:1011660000001FC03FE000601FE03FE0606060607D
:101176007FE03FE00000000000000C0006000300D6
:1011860000001FC03FE000601FE03FE0606060605D
:101196007FE03FE0000000000000060009000600B6
:1011A60000001FC03FE000601FE03FE0606060603D
:1011B6007FE03FE0000000000000000000000000AB
:1011C60000001F803FC070E060006000600070E0BB
:1011D6003FC01F8006001E00000006000F00198099
:1011E60000001F803FC070607FE07FE0600060000D
:1011F6003FC01F8000000000000000001980198019
:1012060000001F803FC070607FE07FE060006000EC
:101216003FC01F800000000000000C000600030015
:1012260000001F803FC070607FE07FE060006000CC
:101236003FC01F8000000000000000001B001B00D4
:1012460000000E000E00060006000600060006005E
:101256001F801F8000000000000006000F0019809C
:1012660000000E000E00060006000600060006003E
:101276001F801F800000000000000C000600030015
:1012860000000E000E00060006000600060006001E
:101296001F801F80000000001980198000000600D2
:1012A60006000F000F001980198030C03FC07FE094
:1012B6006060606000000000060009000600000093
:1012C60006000F000F001980198030C03FC07FE074
:1012D60060606060000000000180030006007FE09F
:1012E6007FE0600060007F807F80600060006000BB
:1012F6007FE07FE00000000000000000000000002A
:10130600000000003DC0666006603FC066006600E3
:1013160066603BC00000000007E007E00F000F001A
:101326001F001B001BC033C033003F007F0063005B
:1013360063E063E000000000000006000F00198073
:1013460000001F803FC070E060606060606070E019
:101356003FC01F80000000000000000019801980B7
:1013660000001F803FC070E060606060606070E0F9
:101376003FC01F800000000000000C0006000300B4
:1013860000001F803FC070E060606060606070E0D9
:101396003FC01F8000000000000006000F001980FB
:1013A600000060606060606060606060606070E067
:1013B6003FE01F600000000000000C000600030074
:1013C600000060606060606060606060606070E047
:1013D6003FE01F6000000000000000001980198037
:1013E600000030C030C0198019800F000F000600C1
:1013F60006000C000C0018001980198000001F80E0
:101406003FC070E06060606060606060606070E077
:101416003FC01F80000000000000000019801980F6
:10142600000060606060606060606060606070E0E6
:101436003FE01F6000000000000000000000000008
:1014460000001F603FC071E0636066606C6078E01A
:101456003FC06F80000000000000000007800FC042
:101466000CC00C000C001F000C000C0018003FE024
:101476003BC0000000000000000000001F603FC0ED
:1014860071E063606360666066606C606C6078E003
:101496003FC06F8000000000000000000000000058
:1014A60030C019800F0006000F00198030C0000000
:1014B6000000000000000000038007C006C0060010
:1014C6000600060006001F8006000600060006004D
:1014D60036003E001C0000000000030006000C0061
:1014E60000001FC03FE000601FE03FE060606060FA
:1014F6007FE03FE0000000000000030006000C0053
:1015060000000E000E00060006000600060006009B
:101516001F801F80000000000000030006000C0072
:1015260000001F803FC070E060606060606070E037
:101536003FC01F80000000000000030006000C00F2
:10154600000060606060606060606060606070E0C5
:101556003FE01F6000000000000000000EC01B807E
:1015660000003F803FC030E0306030603060306067
:1015760030603060000000000EC01B80000060601C
:10158600706078607C606E60676063E061E060E078
:1015960060606060000000001FC03FE000603FE048
:1015A6007FE060607FE03FE000003FC03FC000009A
:1015B60000000000000000001F803FC070E0606077
:1015C600606070E03FC01F8000003FC03FC0000069
:1015D60000000000000000000600060000000600F3
:1015E600060006000E001C0038007060606070E0A7
:1015F6003FC01F8000000000000000001FC03FE049
:1016060070706F306DB06F306DB06DB070703FE060
:101616001FC0000000000000000000000000FFE006
:10162600FFE00060006000600060006000000000F5
:101636000000000000000000000000003000700004
:1016460030C031807B0006000DC0186030C00180BC
:1016560001E0000000000000000000003000700003
:1016660030C031807B0006000D601B6033E00060F7
:1016760000600000000000000600060000000000F8
:101686000600060006000F000F000F000F000F00F7
:101696000600060000000000000000000000000038
:1016A600000018C031806300318018C000000000BF
:1016B6000000000000000000000000000000000024
:1016C60000006300318018C0318063000000000014
:1016D6000000000000000000888022208880222070
:1016E60088802220888022208880222088802220CC
:1016F60088802220888022205550AAA05550AAA072
:101706005550AAA05550AAA05550AAA05550AAA017
:101716005550AAA05550AAA07770DDD07770DDD0BD
:101726007770DDD07770DDD07770DDD07770DDD063
:101736007770DDD07770DDD0060006000600060063
:101746000600060006000600060006000600060063
:101756000600060006000600060006000600060053
:10176600060006000600FE00FE0006000600060053
:101776000600060006000600030006000C00060030
:1017860006000F000F001980198030C03FC07FE0AF
:10179600606060600000000006000F00198006000F
:1017A60006000F000F001980198030C03FC07FE08F
:1017B60060606060000000000C0006000300060088
:1017C60006000F000F001980198030C03FC07FE06F
:1017D6006060606000000000000000001FC03FE085
:1017E600707067306DB06C306DB0673070703FE010
:1017F6001FC000000000000036003600360036002C
:1018060036003600F600F6000600F600F600360052
:101816003600360036003600360036003600360012
:101826003600360036003600360036003600360002
:1018360036003600360036000000000000000000CA
:1018460000000000FE00FE000600F600F60036006E
:1018560036003600360036003600360036003600D2
:1018660036003600F600F6000600FE00FE00000018
:1018760000000000000000000000060006000F80C7
:101886001FC03EC03600360036003EC01FC00F8067
:1018960006000600000000006060606030C030C0D6
:1018A600198019800F000F0006003FC006003FC0D8
:1018B6000600060000000000000000000000000016
:1018C600000000000000FE00FE0006000600060004
:1018D60006000600060006000600060006000600D2
:1018E60006000600060007F007F0000000000000F2
:1018F60000000000000000000600060006000600CA
:10190600060006000600FFF0FFF0000000000000E1
:1019160000000000000000000000000000000000C1
:10192600000000000000FFF0FFF0060006000600C1
:101936000600060006000600060006000600060071
:1019460006000600060007F007F00600060006007F
:101956000600060006000600000000000000000069
:10196600000000000000FFF0FFF000000000000093
:101976000000000000000000060006000600060049
:10198600060006000600FFF0FFF00600060006004F
:101996000600060006000600000000000EC01B80C0
:1019A60000001FC03FE000601FE03FE06060606035
:1019B6007FE03FE0000000000EC01B800000060034
:1019C60006000F000F001980198030C03FC07FE06D
:1019D60060606060000000003600360036003600A9
:1019E6003600360037F037F030003FF03FF00000A9
:1019F60000000000000000000000000000000000E1
:101A0600000000003FF03FF0300037F037F03600BE
:101A16003600360036003600360036003600360010
:101A260036003600F7F0F7F00000FFF0FFF0000098
:101A360000000000000000000000000000000000A0
:101A460000000000FFF0FFF00000F7F0F7F03600AE
:101A560036003600360036003600360036003600D0
:101A66003600360037F037F0300037F037F0360002
:101A76003600360036003600000000000000000088
:101A860000000000FFF0FFF00000FFF0FFF0000094
:101A96000000000000000000360036003600360068
:101AA60036003600F7F0F7F00000F7F0F7F03600F2
:101AB6003600360036003600000060606F603FC0BA
:101AC60070E0606060606060606070E03FC06F60A2
:101AD6006060000000000000000000000F001F8092
:101AE600188018001C000E0007000F80198019804E
:101AF6001F800F00000000003F003F8031C030C053
:101B060030603060786078603060306030C031C0FE
:101B16003F803F000000000006000F0019807FE0B4
:101B26007FE0600060007F807F8060006000600072
:101B36007FE07FE0000000001980198000007FE050
:101B46007FE0600060007F807F8060006000600052
:101B56007FE07FE00000000018000C0006007FE038
:101B66007FE0600060007F807F8060006000600032
:101B76007FE07FE00000000000000600060006008F
:101B8600060006000600000000000000000000003D
:101B960000000000000000000180030006001F8016
:101BA6001F80060006000600060006000600060066
:101BB6001F801F800000000006000F0019801F8094
:101BC6001F80060006000600060006000600060046
:101BD6001F801F80000000001980198000001F80F0
:101BE6001F80060006000600060006000600060026
:101BF6001F801F8000000000060006000600060089
:101C0600060006000600FE00FE00000000000000C0
:101C160000000000000000000000000000000000BE
:101C260000000000000007F007F0060006000600AE
:101C36000600060006000600FFF0FFF0FFF0FFF0CA
:101C4600FFF0FFF0FFF0FFF0FFF0FFF0FFF0FFF016
:101C5600FFF0FFF0FFF0FFF00000000000000000C2
:101C66000000000000000000FFF0FFF0FFF0FFF0B2
:101C7600FFF0FFF0FFF0FFF006000600060006008A
:101C86000600060000000600060006000600060024
:101C9600060006000000000018000C0006001F8069
:101CA6001F80060006000600060006000600060065
:101CB6001F801F8000000000FFF0FFF0FFF0FFF024
:101CC600FFF0FFF0FFF0FFF0000000000000000052
:101CD60000000000000000000180030006001F80D5
:101CE6003FC070E06060606060606060606070E08F
:101CF6003FC01F8000000000000000000000000040
:101D06000F00198030C030C03F8031C030C030C0B5
:101D160031C03F803000300006000F0019801F8060
:101D26003FC070E06060606060606060606070E04E
:101D36003FC01F800000000018000C0006001F8036
:101D46003FC070E06060606060606060606070E02E
:101D56003FC01F8000000000000000001D8037000B
:101D660000001F803FC070E060606060606070E0EF
:101D76003FC01F80000000000EC01B8000001F80B7
:101D86003FC070E06060606060606060606070E0EE
:101D96003FC01F800000000000000000000000009F
:101DA60060C060C060C060C060C071C07FC07EC0DF
:101DB6006000600060006000000000003C003C0025
:101DC60018001F801FC018C018C01FC01F80180031
:101DD6003C003C00000000003C003C0018001F8056
:101DE6001FC018C018C018C018C01FC01F80180018
:101DF6003C003C000000000001800300060060601B
:101E0600606060606060606060606060606030C09C
:101E16003FC01F800000000006000F0019806060B0
:101E2600606060606060606060606060606030C07C
:101E36003FC01F800000000018000C000600606014
:101E4600606060606060606060606060606030C05C
:101E56003FC01F800000000000000000018003005A
:101E6600060030C030C0198019800F000F00060030
:101E760006000C000C0018000180030006006060DC
:101E860030C019800F000600060006000600060096
:101E96000600060000000000000000000780078022
:101EA600000000000000000000000000000000002C
:101EB6000000000000000000030006000C00000007
:101EC600000000000000000000000000000000000C
:101ED60000000000000000000000000000000000FC
:101EE600000000001F801F800000000000000000AE
:101EF60000000000000000000000000000000000DC
:101F0600060006001F801F800600060000001F80D6
:101F16001F8000000000000000000000000000001C
:101F2600000000001F801F8000001F801F8000002F
:101F36000000000000000000000000007000180013
:101F460030C01980730006000D601B6033E000602E
:101F5600006000000000000000001FE036C066C000
:101F660066C066C036C01EC006C006C006C006C033
:101F760006C006C00000000000001F8030C0300010
:101F860030001F8030C030C01F8000C000C030C08D
:101F96001F8000000000000000000000000000009C
:101FA6000600060000003FC03FC000000600060015
:101FB600000000000000000000000000000000001B
:101FC6000000000013000F000000000000000000E9
:101FD60000000000000000000F001F80198019801B
:101FE6001F800F000000000000000000000000003D
:101FF60000000000000000000000000000000000DB
:1020060000000000108039C039C0108000000000B8
:1020160000000000000000000000000000000000BA
:102026000000000002000700070002000000000098
:10203600000000000000000018003800180018001A
:102046001800000000000000000000000000000072
:1020560000000000000000003C0006001C00060016
:102066003C0000000000000000000000000000002E
:1020760000000000000000003C0006001C003000CC
:102086003E0000000000000000000000000000000C
:10209600000000000000000000000000000000003A
:1020A6000F000F000F000F000F000F0000000000D0
:1020B600000000000000000000000000000000001A
:1020C600000000000000000000000000000000000A
:1020D600000000000000000000001E0060077E07F0
:1020E60000F01EF060F77EF7FBDE1F00E007FF073B
:1020F60000F81FF8E0FFFFFF00001E0060077E07E4
:1021060000F01EF060F77EF7FBDE1F00E007FF071A
:1021160000F81FF8E0FFFFFF03004A0053004A00E3
:10212600A3004A00030072007B0072000300EA006D
:1021360003009A0053009A000300EA0000004000E2
:102146008000C00000014001A00050000000000017
:10215600A000A000500000000000F8000000FF00F2
:102166000000FF0000007F80001E0F80007FE7C098
:10217600007FFFE0003FFFE00007FFC00001FFC057
:102186000001FF800001FF0003FFFE0007FFFC00C7
:1021960007FFF00003FFF00003FFFE00001FFFC073
:1021A60001FFFFF001FFFFF801FFFFF8007FFFF8D6
:1021B6000007FE00003FFF00007FFF80007FFF80DA
:1021C600007FC100001FE000001FF000001FF000AC
:1021D600000FE0000007C0000007C0000007C000B5
:1021E600000780000003000000030000000200005A
:1021F60000000000000000000000E00000000000F9
:102206000003900000000000000E1800000000000F
:10221600003808000000000000C0180000000000A0
:1022260003807000000000000C01C0000001800661
:10223600300700000003C00F401C00000006E01D30
:10224600C0700000000C3039C1C0000000181871C1
:10225600C7180000001C0CE1DC7C0000000E07C360
:10226600F1C4000000070386070600000003800E85
:102276001C0200000001C01C300300000000E03812
:1022860018010080000070700FC183C0000038E0A4
:1022960003E08E6006001DC00020FC200F000F80AA
:1022A60000307030198007000010003030C0000088
:1022B600001800E060600000000803806030000045
:1022C600000C0E003018000000043800180C000046
:1022D6000006E0000C060000000380000603000074
:1022E6000000000003018000000000000180C00023
:1022F6000000000000C0C000000000000060C00038
:10230600000000000030C000000000000030C000E7
:10231600000000000030C000000000000030C000D7
:10232600000000000030C000000000000030C000C7
:10233600000000000030C000000000000030C000B7
:10234600000000000030C000000000000030E00087
:10235600000000000030700000000000003018008F
:102366000000000000300C000000000000300400F7
:1023760000000000003FFC0000000000003FFC00E1
:10238600436F6C6F72546F75636820567320312EDD
:1023960032392000426C6F636B200043616C6962C6
:1023A600726174696F6E004F4B00253032580025FC
:1023B600303458002533642E2530326400253564C8
:1023C600002564002532640025336400444400007F
:1023D600256400253032580025313064004F4E0008
:1023E600426C6F636B0077616C6C610001002D4E6F
:1023F600414E00000100D70BF2230000F894EE27AF
:10240600ECBBF1E0F5BFE5BFE0936C00F8E1F1BD90
:10241600E1BD8DE0A2E0BB27ED938A95E9F780E068
:1024260090E1A0E0B1E0ED930197E9F7EAEFF3E27E
:1024360085919591009761F0A591B59105901590BC
:10244600BF01F00105900D920197E1F7FB01F0CF76
:10245600EFEFEDBFE0E1EEBFC0E0D3E00C94C515B1
:10246600E881E03011F01C9A01C01C983CC00E9423
:10247600EE2C0E94EE2C0E94F32CFA93EA93EFE3E3
:10248600F0E00E94F82C08950E940B2A0E94692A07
:102496000E94FE2C0E94EE2C0E94042D0E941B1A04
:1024A600E6E8F3E20E94092DE0910B03E05DEA9372
:1024B6000E94131A0E94EE2C0E940D2D0E941B1AD8
:1024C600EAE9F3E20E94092D0E94122DEA930E9486
:1024D60004170895E881E064E7B9369A349BFECF85
:1024E600349AE4B1F5B121960895E881F981AA817B
:1024F600BB81AE17BF071CF4EA1BFB0B06C0A88105
:10250600B981EA81FB81EA1BFB0B24960895289783
:102516000E9447350E94172DE0938F06F093900690
:10252600E0919B06F0919C06E0938D06F0938E0653
:102536000E941C2DE0938B06F0938C06E091990681
:10254600F0919A06E0938906F0938A060E94212D5F
:10255600E0E00E94282DA0919B06B0919C06A03930
:10256600E1E0BE07ECF4EFE0E0936100E1E00E94F9
:10257600302DE5E00E94372DE1E00E94282DEFE0A6
:10258600E0936100E8E00E94302DEAE00E94372DDA
:10259600E0E0EA939FDFE0939906F0939A060AC07B
:1025A600E0E0F0E0E0939906F0939A06E0939B064C
:1025B600F0939C060E94212D0E941C2DA0918B0653
:1025C600B0918C06EA0FFB1FA0919906B0919A066E
:1025D6000E943E2D8F010E94172DA0918F06B0916B
:1025E6009006EA0FFB1FA0919B06B0919C060E94E5
:1025F6003E2D9F01E0918B06F0918C060E94452DA1
:10260600FF93EF930E941C2D0E94452DAF91BF9121
:10261600EA0FFB1FFF93EF93E0919906F0919A065C
:102626000E94452DAF91BF91EA0FFB1FE0939506DF
:10263600F0939606E0918F06F09190060E944B2D3E
:10264600FF93EF930E94172D0E944B2DAF91BF91E0
:10265600EA0FFB1FFF93EF93E0919B06F0919C0618
:102666000E944B2DAF91BF91EA0FFB1FE093970697
:10267600F0939806A0919506B0919606E4E1F0E0F5
:102686000E94BA320E2EA0919706B0919806E4E108
:10269600F0E00E94BA32E02931F0E0E0E887E9870D
:1026A600EA87EB87B8C000939106109392062093B1
:1026B6009306309394060E94512D989724F40E9415
:1026C600562D98970CF023C0E0E0F0E0E0938106E9
:1026D600F0938206E0917906F0917A06309769F4D4
:1026E6000E945B2D0E94632D1B9734F0E1E0F0E021
:1026F6000E94682D0E946D2D0AC0E230A0E0FA0704
:1027060021F0E330A0E0FA0711F40E9448190E9474
:10271600512D999724F00E94562D99970CF47BC061
:10272600A1E8B6E00E94742DA0917906B0917A06D0
:102736000E94413514F00C940E140E947A2D0E94CA
:10274600512D0E947F2D0E94862D0E948B2DE0EF39
:10275600F0E060E070E00E94ED327F936F93FF93AC
:10276600EF930E94902D0F010E947A2DDF01F00158
:10277600EA1BFB0BAF91BF918F919F910E94B532DF
:102786000E943D330E94862D0E94952D0E94562D53
:102796000E947F2DEC83FD836E837F83AC81BD8198
:1027A6008E819F81E0E4F1E060E070E00E94ED320E
:1027B6007F936F93FF93EF930E949A2D0F010E94D0
:1027C600952DDF01F001EA1BFB0BAF91BF918F91B5
:1027D6009F910E94B5320E943D33EC83FD836E8348
:1027E6007F83E885F985E0937506F0937606EC819C
:1027F600FD81E0937706F0937806E0917506F091F7
:102806007606FA93EA93E0917706F0917806FA93C2
:10281600EA930E94CB180E944E350C9402170E9430
:10282600421AE2E0E09301030E949F2D0E949F2D31
:102836000E94361AE1EAF3E20E94092DE4E1EA93E6
:102846000E94A416E0E9F1E00E94A42DE4E1EA93D7
:102856000E94A4160E94A82D0E94413514F4A89542
:10286600F9CFE2E0E09300030E94EE2C0E94AD2D2A
:102876000E94361AEBE10E94B22D0E94A82D5F97A6
:1028860014F4A895FACF0E94B92DA0E0B0E00E94FA
:10289600C22DEAE5F0E00E94C52D0E947A2D0E9425
:1028A600C92D0E94A82D5E9714F0A895FACF0E9414
:1028B600EE2C0E94AD2D0E94CD2DE2E0E0930003A8
:1028C6000E94D42D0E94361AEAE10E94B22D0E947F
:1028D600A82D5F9714F4A895FACF0E94B92DA2E00F
:1028E600B0E00E94C22DE2E8F0E00E94C52D0E94F1
:1028F600902D0E94C92D0E94A82D5E9714F0A895D0
:10290600FACF0E94D42D0E94CD2D0E94D92D0E946F
:10291600EE2C0E94361AE8E10E94B22D0E94A82DE4
:102926005F9714F4A895FACF0E94E12DA4E0B0E0D9
:102936000E94C22DEAEAF0E00E94C52D0E94952D64
:102946000E94C92D0E94A82D5E9714F0A895FACF73
:10295600E9E6F0E0FA93EA930E94EE2C0E94CD2D70
:102966000E94D92DEEE1F1E00E94C52DE9E10E9419
:10297600B22D0E94A82D5F9714F4A895FACF0E9455
:10298600E12DA6E0B0E00E94C22DE2EDF0E00E944B
:10299600C52D0E949A2D0E94C92D0E94A82D5E97D2
:1029A60014F0A895FACFE9E6F0E0FA93EA93EEE19F
:1029B600F1E0FA93EA930E94CD2D0E949F2DEAEF53
:1029C600F0E00E94C52DEDEAF3E20E94092DE0ED4C
:1029D600F7E00E94A42D0E94421A08950E94EA2D53
:1029E600E4E6E2BF78940E94881891DDA091200861
:1029F600A13028F0E0912008E150E0932008E09112
:102A06001F08E0931E08E6B3AFEFEA27E0931F081E
:102A1600E03019F0E3E0E0932108E0911F08A0916F
:102A26001E08EA17A9F4A0911F08A03021F0A09172
:102A36002008A03069F0A0911F08A03041F4A091B1
:102A46002008A03021F4A0912108A03009F40FC07D
:102A5600F894E091FD06E160E093FD067894E2E3E8
:102A6600E0932008E0912108E150E0932108ACE1D1
:102A7600B8E00E94742DE091FE03EF5FE093FE0341
:102A8600A091FE03AE3149F4A091FD03E3E8EA27E5
:102A9600E093FD03E0E0E093FE0308C00E94EA2D08
:102AA6001A93E6E0E4BD0E949C291991E991EFBFD3
:102AB600F991E991B991A991999189917991699140
:102AC600F9901990099018951A93A895C1D1E130FB
:102AD60011F00C94AC15E091E506E1501E2FA09183
:102AE600E406A13021F40E94F82DE03009F412C06A
:102AF6000E94F82DE093FA06E1E0E093FD060E94BD
:102B0600FF2DBF010E94FF2DE081E260DB01EC9307
:102B16000E94052EA091E406A23011F0A430C9F45B
:102B26000E94F82DE093FB06E5E1E093FA06E1E06A
:102B3600E093FD060E94F82DE03029F00E94FF2D5B
:102B4600E081E27009F405C01A93E2E0EA930E947C
:102B5600A31AE091FD03E07889F0E091FD03EF7799
:102B6600E093FD030E94451DE091FD03E07131F005
:102B7600E091FD03E270EA930E947B190E94A1276F
:102B860019910895E0E0E5BFE0936D00E0936C00D5
:102B9600EBBBEFEFEABBE0E0E8BBE7BBE5BBEFEF83
:102BA600E4BBE0EFE2BBE1BBE0E3E3B9ECEBE2B9A7
:102BB600E0E0E0936200E0936100EFE0E0936500FF
:102BC600E0936400E0E0E0BFE7E0E3BFE4E6E2BFF5
:102BD600E0E0E1BFEFBDEEBDEDBDECBDE7BDE6BD9E
:102BE600EBBDEABDE9BDE8BDE0937900E09378006E
:102BF600E3E0E5BDE6E0E4BDE0E0E3BDE0938B00A5
:102C0600EAE0E0938A00E0E0E0938900E093880040
:102C1600E0938100E0938000E2E1E0938700E4E343
:102C2600E0938600E0E0E0938500E0938400E09383
:102C36008300E0938200E0936A00E0E3EABFE0E409
:102C4600E9BFE8BFE1E4E7BFE0E0E0937D00EBB970
:102C5600E8EDEAB9E6E0E0939500E0E0E093900065
:102C6600E7E6E9B9E0E0E0939B00E8EDE0939A003F
:102C7600E6E0E0939D00E0E0E0939800E3E3E09374
:102C86009900E0E8E8B9E0E0E0BDE0E4E7B9E7E8AC
:102C9600E6B9E0B5EF7EE0BDE0E2E0937000E0E08B
:102CA600E0937200E4E4E0937400EFE1E1BDEFE04D
:102CB600E1BD78940E94D62515D3E1E0EA930E94FF
:102CC60033120E94122DE53128F0A8E0B0E0E4E1CD
:102CD6000E94B0330E94471221E0E5E1E093FA0634
:102CE6000E947A2D0F010E94902D0E161F0644F4A5
:102CF6000E94952D0F010E949A2D0E161F060CF0AC
:102D06008EDDE1E0EA931DD000E010E00436E0E05D
:102D16001E0724F40E94A127E03009F005C00E9496
:102D26000A2E0F5F1F4FF2CF0436E0E01E0734F085
:102D36000E94A82D5F9714F00E941214C5DEFECFE4
:102D4600FFCFE881E03021F4EAEAF0E00E940D2EA0
:102D5600A881A13021F4E4EAF0E00E940D2EA881BA
:102D6600A23021F4E0EBF0E00E940D2EA881A33002
:102D760021F4EEEBF0E00E940D2EA881A43021F4A0
:102D8600E4ECF0E00E940D2E51C31A9310E00E946D
:102D9600122EE03031F00E94122EEA9341D31F5FCB
:102DA600F6CF1881239608951A930A93E0E0E093EC
:102DB6009D06E0939E0610E0143190F400E0033087
:102DC60068F4A3E01A9FF001EC55F94FDF01EE27F6
:102DD600A00FBE1FE0E2EC930F5FF1CF1F5FECCFB9
:102DE600D4C12A970E94192EE3ECF3E2FA93EA93F0
:102DF600EE85FF850E94B5320E941D2EC6DF2C96F9
:102E060008952A970E94192EEAECF3E2FA93EA93C0
:102E1600EE85FF27662777270E941D2EB6DF2B96A5
:102E260008951A930A9300E010E00E94242EE030E1
:102E360021F00832E0E01E070CF007C00E94242EA5
:102E4600EA93EED20F5F1F4FF0CF1981088115C3A9
:102E5600E091E306A091E206EA17C1F00E942B2E4C
:102E6600AE0FBF1FEC91E093E5060E942B2EEA0FF2
:102E7600FB1FE181E093E406A091E306AF5FEAE081
:102E86000E944233E093E306E1E00895E0E008950E
:102E96000E94332EA981A0830E94332E3196A881E9
:102EA600A083A091E206AF5FEAE00E944233E0937E
:102EB600E206B4C21A930E943D2EE45FFC4FA0E0E6
:102EC600A0830E943D2EEA5EFC4F108117FF05C0CD
:102ED600E12F0E94422EA0E0A08316FF05C0E12F3D
:102EE6000E94492EA0E0A0830E943D2EEA5EFC4F80
:102EF600A0E0A0830E943D2EEB5EFC4FA0E0A083E5
:102F060018818CC2AD970E944535EAADFBADAEADDA
:102F1600BFADEA0FFB1FAF0110E0143188F50E9428
:102F2600F82DE03041F10E94502EDF010E947833E7
:102F3600DF01ECADFDADEA17FB07E9F40E94562E62
:102F4600DF01EEADFFADAE17BF07ACF00E94562E07
:102F56004E175F0784F00E945F2EAE0FBF1FEEADC7
:102F6600FFADAE17BF073CF00E945F2EAE0FBF1F2E
:102F76004A175B070CF402C01A939CDF1F5FCDCF84
:102F860010E0143110F00C9482180E94F82DE030F5
:102F960011F00C948018ACE01A9FF001E45FFC4F2E
:102FA600AFA90E946E2EE35FFC4FAEADBFADA0830E
:102FB600B1830E94502EACADBDADA083B183ACE011
:102FC6001A9FF001EF5EFC4FAAAD0E946E2EEE5ED8
:102FD600FC4FA8AD0E946E2EED5EFC4FA091020341
:102FE6000E946E2EEC5EFC4FA0910303A0830E940C
:102FF600FF2D0F01E091FC03E295E07FA091040311
:10300600EA0FD001EC930E94732EA0E00E946E2E70
:10301600E95EFC4FA0E0A083E0E0EE83EDA9FEA907
:10302600309741F00E94792EEFA9F8ADFA93EA9312
:103036000E94992AEBA9FCA9309731F00E94792EBB
:10304600EDA9FEA90E947E2EE0E0EEA70E94792E51
:103056000E94A42A3E2F3B30A8F000E00E94822E58
:1030660011F00C3008F002C00F5FF8CF0E94822EDC
:1030760049F40E948A2E30E00E94732EDF01E02F71
:10308600E058EC93E0E0E88B3130F0F000E00E948D
:10309600942E11F00C3008F002C00F5FF8CF0E949A
:1030A600942E91F4ABE00A9FF001EB5FFB4FFA938D
:1030B600EA93FE0138960E947E2E30E00E94732E1F
:1030C600DF01E02FE05CEC933130A8F000E00E94D5
:1030D600822E11F00C3008F002C00F5FF8CF0E946C
:1030E600822E49F40E948A2E30E00E94732EDF0160
:1030F600E02FE058EC93E12F03C01F5F42CFEFEFC4
:103106000E944C35EF96219608951A930A930E94D1
:103116009C2E3097D1F1E0917B06F0917C0630979A
:1031260069F50E949C2E0E948233E0937B06F09301
:103136007C06309731F4E0E0F0E00E940D2EE0E0EE
:103146001AC00E94A12E0E949C2E0E948233F595E1
:10315600E7958F01D801E0E0F1E00E941333E09398
:103166008700D801E0E0F1E00E944533E093860055
:103176000E94A12EE0E4E0938B0007C0ABE7B6E027
:10318600ED91FD913197FE93EE9309911991089572
:103196001A930A9300E010E0143110F00C94111900
:1031A6000E94F82DE030C1F10E94562EAC81BD81FF
:1031B600EA17FB0764F50E94502EDF010E94783360
:1031C600AA81BB81EA17FB0714F5ACE01A9FF00150
:1031D600E35FFC4F608171811A9FF001EF5EFC4F47
:1031E6000E94A92EAC81BD81AE17BF0784F40E9450
:1031F600502E60817181ACE01A9FF001EE5EFC4FAB
:103206000E94A92EAA81BB81AE17BF070CF004C08D
:10321600E12FEF5F0E2F02C01F5FBECF003081F09F
:10322600E0918306F0918406A02FB0E0EA17FB0731
:1032360031F0A0918306B0918406109709F401C07D
:103246001FC00E94632DD29714F40E945B2D0E942A
:10325600632D1397A1F40A93E1E0EA9319DEE02FB8
:10326600F0E0E0938306F0938406E02FF0E0E0932D
:103276008706F0938806E2E0F0E00E94682D01C020
:1032860004D01981088126960895E0918306F0916D
:103296008406309701F10E94632D999734F4E091EA
:1032A6008306EA93E2E0EA93F3DD0E94632D9997A1
:1032B60034F0E0918306EA93E4E0EA93E9DDE0E0A6
:1032C600F0E00E94682D0E946D2DE0E0F0E0E093B2
:1032D6008306F0938406E0E0F0E0E0938706F0933F
:1032E60088060895CCD060DDE5E1E093FA060895FE
:1032F6000E944535A0919F06A43120F4A091A00616
:10330600A33008F032C0E0919F060E94AE2E8F01D6
:10331600E091A006F0E0A4E1B0E00E94E8329F014F
:103326000E94B42EECE0F0E0FA93EA930E94B92EE4
:103336000E94A7320E94F82CEE81E030B1F0E091B5
:103346009F06A3E0EA9FF001EC55F94FDF01E091FB
:10335600A006F0E0AE0FBF1F4C9155270E94B42E79
:103366004A93E0E0EA930E9465260E944C35279630
:1033760008950E94F32CA0910703B0910803AE179D
:10338600BF075CF4E0910104F0910204A0910903E7
:10339600B0910A03AE17BF070CF040C0E0910703D7
:1033A600F0910803FA93EA93E0910903F0910A0376
:1033B6000E94BD2E0E946526A0917D06B0917E06D4
:1033C600549734F4A0917F06B091800613970CF0C1
:1033D60012C0E0917D06F0917E06A3E0B0E00E9467
:1033E600C032EC55F94FA0917F06B0918006EA0FE6
:1033F600FB1FA981A0830E94C42EA0910703B09150
:1034060008030E94CA2E0E94CE2EE0917D06F091FE
:103416007E063196E0937D06F0937E062296089509
:10342600E881EA93E0910303EA93A3DF21960895E6
:10343600EA81FB81E0937D06F0937E06E881F981BF
:10344600E0937F06F0938006AA81BB81ECE0F0E072
:103456000E94E8320E94CE2EA881B981E4E1F0E014
:103466000E94E83206C0EA81FB810E94CE2EE881E6
:10347600F981E0930903F0930A03249608950E94C4
:10348600D32E143120F41A9315DD1F5FFACF0E9454
:10349600EE2C0E94EE2C0E94F32CFA93EA93E09114
:1034A6000104F09102040E94F82C10E01C3048F44C
:1034B600A9E21A9FF001E757FB4FA0E0A0831F5F28
:1034C600F5CF10E01C3048F4ABE01A9FF001EB5F3B
:1034D600FB4FA0E0A0831F5FF5CFE091FD03EF7ED9
:1034E600E093FD03E5C20E94D32E1431C0F40E947E
:1034F600502E0E94DB2EAE17BF0764F00E94502E9E
:103506000E94E22EEA17FB072CF00E94732EE08140
:10351600E03009F402C01A93CDDC1F5FE6CF0E94AB
:10352600EE2CED81FE81FA93EA930E94F32CFA9336
:10353600EA93A985BA850E94E92E0E94F82C9FC2BB
:10354600EE970E9445350E94EE2EE03009F460C2E7
:103556000E94EE2EEFAFE07851F00E94792EFE0128
:10356600EF5BFF4FE0810E94422E0E947E2EEFAD60
:10357600E07451F00E94792EFE01EF5BFF4FE0816F
:103586000E94492E0E947E2E0E94792E0E94A42A15
:10359600EEAFE0910003E9AFE0910103E8AF0E94CE
:1035A600FE2C0E94F92EE35FFC4F008111810E94E0
:1035B600F92EE15FFC4F208131810E94F92EEF5EEA
:1035C600FC4F408155270E94F92EEE5EFC4FE081AC
:1035D600F0E0DE01AE5BBF4FED93FC930E94F92E47
:1035E600ED5EFC4FE081EAAF0E94012FDF010E94F1
:1035F600B92E0E94E8320E94062F0E94B42E5A93DA
:103606004A930E940C2FFA93EA93FE01EE5BFF4F5A
:10361600E081EA930E940D260E94B42E0E94132F89
:103626003A932A930E94192F0E941D2F0E94282F39
:103636000E942B2F0E94F92EEB5EFC4FE081E07179
:1036460081F00E94B42E5A934A930E94042D0E9440
:10365600312FFA01E00FF11F35970E94352F0E9496
:103666003A2F0E94F92EEB5EFC4FE081E07269F082
:103676000E941D2F36970E94422F0E94042D0E9401
:10368600312F0E94B42E0E943A2F0E94B42E1A9314
:103696000A930E942B2F0E94132F3A932A930E947B
:1036A600132F0E942B2F0E94472FA130B1F41A939B
:1036B6000A93F90131960E94282FF9013196FA935F
:1036C600EA930E94192FF80131960E94352FF801CE
:1036D6003196FA93EA930E942B2F0E94472FA2302D
:1036E600E1F40E941D2F31970E94282F0E940C2F73
:1036F600E20FF31F3197FA93EA930E94192FFA010A
:10370600E00FF11F31970E94352FFA01E00FF11FEC
:103716003197FA93EA930E942B2FFE01EC5BFF4F41
:10372600E081E03011F40C94DF1C0E94F92EEC5E6F
:10373600FC4FE081EAAF0E94C42E0E944C2F0E94EB
:103746001333EBAFAEADEA1710F40C94FB1BE1E0BC
:10375600E0930103E03041F00E94012FEE0FFF1FBE
:1037660034960E944F2F0CF009C0E2E0E09301036B
:103776000E94012FEE0FFF1F0E94062FDE01A05CA4
:10378600BF4F0D90BC91A02D0E94592FEA1BFB0B39
:10379600DF010E94602F0E94652F32F4FE01E05C7B
:1037A600FF4F002401920082AEAD0E946C2F0E9452
:1037B6004C2F0E94742FECAF0E94472FA13021F4AA
:1037C6000E94772F0E947C2F0E94472FA23021F45F
:1037D6000E94772F0E94842FE0E0EFAF0E948A2F8D
:1037E600E03029F00E948A2F0E94922FF7CFE4C082
:1037F600FE01E05CFF4F0190F081E02DEE0FFF1F10
:10380600DE01AE5BBF4F0D90BC91A02DAE1BBF0B72
:10381600E3E0F0E00E9413330E94652F22F4E1E01A
:10382600F0E00E94062FEBADA2E0EA9FF001AEADFC
:10383600AE17A8F5E1E0E0930103E03041F00E9405
:10384600012F0E94AB3236960E944F2F0CF009C012
:10385600E2E0E09301030E94012FEE0FFF1F0E949A
:10386600062FEEADEDAFEDADE150EDAFEDAD0E9443
:103876009B2FA03219F0ADADA13008F404C0EDAD18
:10388600E150EDAFF3CFADAD0E946C2FAE2FFA0134
:10389600B0E0EA17FB073CF3EDADE03011F4EBAD19
:1038A600EDAFADADECE0EA9FF0010E944C2F0E9417
:1038B600742FECAF0E94472FA13021F40E94772F7E
:1038C6000E947C2F0E94472FA23021F40E94772F5E
:1038D6000E94842FE0E0EFAFEFAD0E949B2FA03057
:1038E60021F0EDADAFADAE1708F005C00E948A2FEE
:1038F6000E94922FF1CFEFAD0E949B2FA03221F4B0
:10390600EEADAFADAE1708F007C0EFADEF5FEFAFAE
:10391600EDADEF5FEDAFEFCFADADEEADEA1BAE2F88
:10392600EBADEA1778F0ADADEEADEA1BACE0EA9F81
:10393600F001A0910003EA9FF0010E944C2F0E9423
:10394600742F01C0E0E0ECAF0E94472FA13081F454
:103956000E94772F3196FA93EA930E94012F3197AE
:10396600DF010E94B92E0E94A22F31960E94C52D1A
:103976000E94472FA23071F40E94772FFA93EA93A0
:103986000E94012F3197DF010E94B92E0E94A22FBB
:103996000E94C52DEFAD0E949B2FA03039F0ADAD32
:1039A600EFADEA1BAE2FEBADEA1708F405C00E9497
:1039B6008A2F0E94922FEECF0E94F92EE95EFC4FCD
:1039C600E081E030F9F00E94FE2C0E94B42E4BDD1F
:1039D600E0E0E09303030E94F92EE95EFC4FE081EC
:1039E600EA3040F00E94F92EE95EFC4FE081EA934E
:1039F60008DA08C00E94F92EE95EFC4FE081E05D1E
:103A0600EA930EDDE9ADE0930003E8ADE093010330
:103A16000E944C35EF96279608951A9310E0E89485
:103A260022F8143148F40E94F82DE03011F00E947B
:103A3600052E1F5FA895F5CFE0E0E093030338C09D
:103A46001A9310E01431C0F40E94F82DE03071F0A2
:103A56000E94502E0E94DB2EEA17FB073CF40E94C0
:103A6600502E0E94E22EAE17BF070CF002C00E9435
:103A7600052E1F5FA895E6CFE0E0E09303031881CB
:103A8600259608951A9310E0143190F40E94F82DAB
:103A9600E03029F00E94FF2DE081E17009F406C0B4
:103AA6001A93E091FD03E170EA934ADD1F5FECCFC4
:103AB600199108952C970E944535AD89BE890E94BB
:103AC600602FED8BFE8BAB89BC890E94602FEB8B40
:103AD600FC8BED89FE89A98DBA8DEA0FFB1FE98F54
:103AE600FA8FEB89FC89AF89B88DEA0FFB1FEF8B44
:103AF600F88FED89FE89AD89BE890E94AD2FEE87CC
:103B0600FF87688B798BEB89FC89AB89BC890E941E
:103B1600AD2FAE85BF85888999890E94F834EA87DA
:103B2600FB876C877D8700E010E0EB89FC89E01756
:103B3600F10714F40C94E61DF8010E94B5320E94B8
:103B46002734EE83FF8368877987AE81BF818885B6
:103B560099850E94AA34AA85BB858C859D850E947D
:103B6600AA34AE85BF85888999890E948B330E94C5
:103B76005A340E94F033AF015A934A930E94CF2CD5
:103B86002E2F33270E94B42FE98DFA8DE01BF10BFF
:103B96000E94BB2FED8DFE8DE01BF10B0E94C52F01
:103BA6000E94B42FF801A98DBA8DEA0FFB1F0E945F
:103BB600BB2FF801AD8DBE8DEA0FFB1F0E94C52FEE
:103BC6000F5F1F4FB2CF0E944C356B960895EA8166
:103BD600F0E0EBBBF5BBF7E1F09365001F98E6E17B
:103BE600E0936500F0936500E881F981EBBBF5BBD6
:103BF600FFE1F0936500EEE1E0936500F093650068
:103C06001F9A0C94D421E2E2EBBBE0E0E5BB0C94F6
:103C1600DA210C94E5210E94CB2FEFE1E0936500B9
:103C2600E4E6F0E00E94A42DE5EEEA93E0E0F0E899
:103C36000E94D12FE0E00E94D52FE1E0EA93E0E078
:103C4600F1E00E94D12FE2E0EA93E0E0F4E00E9486
:103C5600D12F0E94D92F0E94DE2FB9DFE8E0EA9328
:103C6600E2E0F2E00E94D12FE9E0EA930E94EE2C16
:103C76000E94EA1DEAE0EA930E94EE2C0E94EA1DE9
:103C8600ECE0EA930E94EE2C0E94EA1DEDE0EA9336
:103C96000E94EE2C0E94EA1DEFE0EA930E94EE2CB1
:103CA6000E94EA1DE0E1EA930E94EE2C0E94EA1DC2
:103CB600E1E1EA930E940D2D0E94EA1DE2E1EA93FA
:103CC6000E94EE2C0E94EA1DE3E1EA930E94EE2C8C
:103CD6000E94EA1D0E949F2D0E948B32E0E1EA932A
:103CE600E0EBFBE10E94D12FE1E1EA930E940D2D6A
:103CF6000E94EA1D0E949F2D0E948B32E2E1EA9308
:103D0600EEE1F1E00E94D12F0E949F2D0E948B329E
:103D1600E3E1EA93E0E0FFE10E94D12FE9E2EA93D2
:103D2600EFE1F0E00E94D12F0E949F2D0E948B327E
:103D3600E0E2EA930E94EE2C0E94EA1DE1E2EA9399
:103D46000E94EE2C0E94EA1DA0910B03A13029F4DB
:103D5600EBE2EA93ECE0F0E004C0EBE2EA93E0E2A7
:103D6600F0E0FA93EA930E94EA1DE0E3EA930E94E8
:103D7600EE2C0E94EA1DE1E3EA930E94EE2C0E94DB
:103D8600EA1DE2E3EA930E94EE2C0E94EA1DE5E3B7
:103D9600EA930E94EE2C0E94EA1DE6E3EA93E1E034
:103DA600F1E00E94D12FE7E30E94E12FE8E30E94B1
:103DB600E12FE9E30E94E12FECE30E94E12FEDE31E
:103DC6000E94E12FE0E5EA930E94EE2C0E94E52F87
:103DD600E2E5EA930E94EE2C0E94EC2FA0910B03E1
:103DE600A13029F4E0E6EA93E0E0F7EA04C0E0E671
:103DF600EA93E0E0F7E2FA93EA930E94EA1DE1E62D
:103E06000E94D52FEAE6EA930E94EE2C0E94EA1D54
:103E1600E0E8EA930E94EE2C0E94EA1DE1E8EA93AC
:103E26000E94EE2C0E94EA1DE2E8EA930E94EE2C24
:103E36000E94EA1DE3E8EA930E94EE2C0E94EA1D26
:103E4600E4E8EA930E94EE2C0E94EA1DE5E8EA9374
:103E56000E94EE2C0E94EA1DE0E9EA93E0E1F0E020
:103E66000E94D12FE2E9EA93E0E0F7E00E94D12F29
:103E7600E3E9EA930E940D2D0E94EA1DE5E9EA9323
:103E8600EFE3F3E00E94D12FE7E9EA930E94EE2CDC
:103E96000E94EA1DE8E9EA930E94EE2C0E94EA1DC0
:103EA600E7E00E94D52F0E949F2D0E948B32E7E00B
:103EB600EA93E1E2F0E00E94D12FE7E0EA93E3E241
:103EC600F0E00E94D12F0E949F2D0E948B32E7E0E6
:103ED600EA93E3E7F1E00E94D12F08950E94F32FC1
:103EE600AE85AA2362F0AD85BE85A03FE0E0BE07A1
:103EF60034F4AB85BC85AF33E1E0BE070CF04EC0B1
:103F06000E940130AE0FBF1FA03FE0E0BE0714F0D5
:103F16000E9406300E940F30AE0FBF1FA034E1E0B2
:103F2600BE0714F00E9414304985E0E50E941D305A
:103F3600E1E50E9421300E942730E2E50E942A3006
:103F4600E3E50E942E300E942730E0E20E941D30F9
:103F5600E1E20E942A3057DE0BBB15BB2EE13FE1A2
:103F660000E010E00E94343064F050E0451730F075
:103F760020936500309365005F5FF8CF0F5F1F4F9A
:103F8600F1CF47DEE0E5EA930E94EE2C0E94E52F92
:103F9600E2E5EA930E94EE2C0E94EC2F52C00E94AA
:103FA600F32F0E940130EA17FB0729F50E943930EA
:103FB60014F40E944030E3E0EA93E8E3F0E10E9463
:103FC600D12FE0E20E941D30E1E20E942A301BDE82
:103FD6000BBB15BB2EE13FE10B851C850E943430DF
:103FE6003CF020936500309365000F5F1F4FF6CFBE
:103FF6000E94D92F24C00E940F30EA17FB0729F52B
:104006000E94513014F40E944030E0E20E941D30BC
:10401600E1E20E942A300E94061E0BBB15BB2EE170
:104026003FE10D851E85E985FA85E017F1073CF02D
:1040360020936500309365000F5F1F4FF4CF0E94F9
:104046000C1E0E944C352F9608950E9458300E94EF
:104056005F30FF93EF930E9463300E945F30AF9111
:10406600BF91EA17FB07D8F10E943930ECF420E043
:1040760030E00E946630E217F307ACF00E94583039
:104086000E946D300E9466300E947230E1E2EA932F
:10409600EC85FD85E21BF30B0E94D12F0E947C303C
:1040A6002F5F3F4FE6CF19C020E030E00E9463301B
:1040B600E217F30794F00E9458300E946D300E9478
:1040C60063300E947230E1E20E9482300E94273003
:1040D6000E947C302F5F3F4FE9CF0C94C8240E948A
:1040E60058300E945F30FF93EF930E9463300E9426
:1040F6005F30AF91BF91EA17FB07E8F50E94513098
:10410600ECF420E030E00E948730E217F307ACF0D1
:104116000E9463300E946D300E9487300E948E306C
:10412600EE85FF85E21BF30B0E94D12F0E9495308E
:104136000E947C302F5F3F4FE6CF1BC020E030E06F
:104146000E945830E217F307A4F00E9463300E94E1
:104156006D300E9458300E948E30F901AE85BF85C1
:104166000E9427300E9495300E947C302F5F3F4F7F
:10417600E7CF0C94C8240C94C82425970E94453593
:10418600EB850E949B300E94A730103110F00C94F2
:104196003A2100E0E09101030E1710F00C94322151
:1041A600E1E20E941D30E0E0EA87AA85A23010F025
:1041B6000C942A210E94B330E252FF4F2491203002
:1041C60011F40C94252127FF34C00E94C530E2E289
:1041D600EBBBE0E0E5BBE7E1E09365001F98F6E1A5
:1041E600F0936500E0936500EE81EBBBEF81E5BBE4
:1041F600EFE1FEE1E0936500F0936500E093650072
:1042060031FF04C0F0936500E093650026FF10C0FF
:10421600F0936500E093650031FF06C0F0936500FA
:10422600E09365004F5F5F4F220F4F5F5F4FEECF0A
:104236001F9A220F31FF02C04F5F5F4F4F5F5F4FE4
:104246000C94E220EA85EF5FEA870C94D820ED858E
:10425600FE853196ED87FE870F5F0C94CD20E885AD
:10426600F9853296E887F9871F5F0C94C8200E946B
:10427600D92F0C94D22523970E944535E9850E94B3
:104286009B303091000310E0EA851E1710F00C9465
:10429600B62100E0E09101030E1710F00C94B32153
:1042A600E1E2EA93ED85FE850E94D12FE0E0E88702
:1042B600EB85A885AE1710F00C94AB210E94CB308D
:1042C600203011F40C94A62127FF34C00E94C5307B
:1042D600E2E2EBBBE0E0E5BBE7E1E09365001F98B7
:1042E600F6E1F0936500E0936500EE81EBBBEF81AC
:1042F600E5BBEFE1FEE1E0936500F0936500E09336
:10430600650031FF04C0F0936500E093650026FF69
:1043160010C0F0936500E093650031FF06C0F0938E
:104326006500E09365004F5F5F4F220F4F5F5F4F61
:10433600EECF1F9A220F31FF02C04F5F5F4F4F5FD4
:104346005F4F0C946321E885EF5FE8870C945B214F
:10435600EC85FD853196EC87FD870F5F0C944D212A
:104366001F5F0C9447210E94D92F0C94D225EA8115
:10437600F0E0E5BBFBBBF7E1F09365001F98E6E1D3
:10438600E0936500F0936500E881F981E5BBFBBB2E
:10439600FFE1F0936500EEE1E0936500F0936500C0
:1043A6001F9A23960895E2E2E5BBE0E0EBBBE7E166
:1043B600E09365001F98E6E1E0936500E7E1E0938E
:1043C600650008951F9A08950E94CB2FEFE1E093B0
:1043D6006500E8ECF0E00E94A42DE6E4EA93E4EA46
:1043E600F0E00E94E030E7E4EA93E3E5F0E00E94C3
:1043F600E030E8E4EA930E94EE2CB9DFE9E4EA93C0
:10440600E4E4F0E00E94E030EAE40E94E430EBE409
:10441600EA93E7E6F0E00E94E030ECE4EA93E3E3B7
:10442600F0E00E94E030EDE4EA93E7E7F0E00E9476
:10443600E030EEE4EA93E2E1F0E00E94E030EFE4FF
:10444600EA93ECE4F0E00E94E030E0E5EA93E6E48B
:10445600F0E00E94E030E1E5EA93E4E4F0E00E9457
:10446600E030E1E0EA930E94042D0E94BA210E9406
:10447600E830E3E2EA93E5E9F0E00E94E030E4E2C6
:10448600EA93E5E9F0E00E94E030E5E2EA93EFEF37
:10449600F0E00E94E030E7E20E94ED30E8E20E94A0
:1044A600ED30E9E20E94ED30EAE20E94ED30ECE206
:1044B6000E94ED30EDE20E94ED30EAE30E94F13019
:1044C600EBE30E94F130ECE3EA93E0EFF0E00E94C8
:1044D600E030EDE3EA930E94EE2C0E94BA21E4E17B
:1044E600F0E00E94A42DE5E3EA93E8E3F0E00E9401
:1044F600E030E6E3EA93E8E7F0E00E94E030EEE33E
:10450600EA93E8E3F0E00E94E030E0E4EA93EFE0CB
:10451600F0E00E94E030E1E4EA93E0EFF0E00E9490
:10452600E030E9E1EA93E9E4F0E00E94E030E3E913
:10453600EA93EFE0F0E00E94E0300E940A2EE0E20B
:10454600EA93E0E4F0E00E94E030EDE1EA930E94B5
:104556000D2D0E94BA21EEE1EA930E94EE2C0E94F4
:10456600BA21EFE10E94E430E4E4EA93EDE4F0E0FE
:104576000E94E030E5E4EA93E1E1F0E00E94E030F9
:104586000E940A2EECE10E94E430E4E1F0E00E9491
:10459600A42DEBE1EA93E8E1F0E00E94E0300E940E
:1045A600F530EBE1EA93E0E1F0E00E94E0300E94B2
:1045B600F530E3E4EA93E0E8F0E00E94E030E4E678
:1045C600F0E00E94A42DE0E9EA93EFE7F0E00E9414
:1045D600E030E6E20E94E4300E94F530E6E2EA933B
:1045E600E4E2F0E00E94E030E6E2EA93ECE2F0E09A
:1045F6000E94E0300E94F530E6E2EA93ECE3F0E058
:104606000E94E030E7E50E94ED30E5E5EA930E947E
:10461600EE2C0E94BA21EEEFEA93EAE5F0E00E9462
:10462600E030E7E5EA930E94EE2C0E94BA21089555
:104636000E94F830AE85AA2362F0AD85BE85A03F04
:10464600E0E0BE0734F4AB85BC85AF33E1E0BE07DE
:104656000CF05DC00E940130AE0FBF1FA03FE0E02E
:10466600BE0714F00E9406300E940F30AE0FBF1F27
:10467600A034E1E0BE0714F00E94143049850E9480
:104686000631E3E0EA93EE85FF850E94E030E4E040
:104696000E9421300E940D31E5E00E942130EA0F90
:1046A600FB1F0E94E0300E941331E7E0EA93EC859D
:1046B600FD850E94E030E8E00E942E300E940D3118
:1046C600E9E00E942E30EA0FFB1F0E94E0306BDE0D
:1046D60005BB1BBB2EE13FE100E010E00E94343039
:1046E60064F050E0451730F0209365003093650084
:1046F6005F5FF8CF0F5F1F4FF1CF64DE0E94DE2FA2
:104706000E941A31E8E00E94F1300E9421313DC139
:104716000E94F8300E940130EA17FB0711F00C9452
:10472600E0230E94393014F40E944030E6E1EA9317
:10473600E8EEF0E00E94E030E4E00E94F130E5E0CF
:10474600EA93EFE3F1E00E94E030E8E0EA930E94AA
:10475600EE2C0E94BA21E9E0EA93EFEEF0E00E9427
:10476600E030E2E0EA93EC85FD850E942631E3E045
:104776000E9429310E942E310E94333114DE05BB7E
:104786001BBB2EE13FE10B851C850E9434303CF0BB
:1047960020936500309365000F5F1F4FF6CF0E9490
:1047A600E5210E94E8300E94DE2F0E941A31E8E0DF
:1047B6000E94F1300E942131E8C00E940F30EA17B2
:1047C600FB0751F50E94513014F40E9440300E94BC
:1047D6000631E3E0EA93EE85FF85F0700E94E03053
:1047E6000E941331E7E00E9429310E94D62105BBC1
:1047F6001BBB2EE13FE10D851E85E985FA85E01795
:10480600F1073CF020936500309365000F5F1F4F62
:10481600F4CF0E94E521B9C00E9458300E945F3053
:10482600FF93EF930E9463300E945F30AF91BF9178
:10483600EA17FB0710F40C946A240E94393034F509
:1048460020E030E00E946630E217F307F4F00E94A1
:1048560058300E946D300E9466300E9439310E94A5
:104866004331E6E0EA93AC85BD85A21BB30BFD019F
:104876000E942631E7E0EA93AC85BD850E944F3160
:104886000E9456312F5F3F4FDDCF20C020E030E041
:104896000E946330E217F307CCF00E9458300E9462
:1048A6006D300E9463300E9439310E944331E6E048
:1048B6000E9482300E940D31E7E00E9482300E9401
:1048C6005C310E9456312F5F3F4FE2CF5EC00E949F
:1048D60058300E945F30FF93EF930E9463300E942E
:1048E6005F30AF91BF91EA17FB0710F00C94C82414
:1048F6000E94513034F520E030E00E948730E21704
:10490600F307F4F00E9463300E946D300E948730F6
:104916000E946331AE85BF85A21BB30BFD010E94C9
:104926002631E3E0EA93AE85BF850E944F310E94AF
:104936006A310E9470310E9456312F5F3F4FDDCFA2
:1049460024C020E030E00E945830E217F307ECF074
:104956000E9463300E946D300E9458300E9463317D
:10496600F901AE85BF850E940D31E3E0EA93F901B6
:10497600AE85BF850E945C310E946A310E9470310B
:104986000E9456312F5F3F4FDECF0E944C352F9647
:10499600089525970E944535EB850E9476310E9441
:1049A600A730103110F00C944C2500E0E091010383
:1049B6000E1710F00C9444250E942E310E943331BC
:1049C600E0E0EA87AA85A23010F00C943C250E940C
:1049D600B330E252FF4F2491203011F40C94372566
:1049E60027FF39C0E2E0EA93FA010E9426310E94CD
:1049F6008231E2E2E5BBE0E0EBBBE7E1E093650094
:104A06001F98F6E1F0936500E0936500EE81E5BB43
:104A1600EF81EBBBEFE1FEE1E0936500F09365000B
:104A2600E093650031FF04C0F0936500E0936500F4
:104A360026FF10C0F0936500E093650031FF06C0C5
:104A4600F0936500E09365004F5F5F4F220F4F5F65
:104A56005F4FEECF1F9A220F31FF02C04F5F5F4FAD
:104A66004F5F5F4F0C94EF24EA85EF5FEA870C9463
:104A7600E524ED85FE853196ED87FE870F5F0C9464
:104A8600D924E885F9853296E887F9871F5F0C9463
:104A9600D4240C94D22523970E944535E9850E949B
:104AA60076313091000310E0EA851E1710F00C9461
:104AB600D22500E0E09101030E1710F00C94CF25EB
:104AC600E6E0EA93ED85FE850E942631E7E0EA936B
:104AD600ED85FE85F0700E94E030E0E0E887EB852A
:104AE600A885AE1710F00C94C7250E94CB30203055
:104AF60011F40C94C22527FF39C0E2E0EA93FA01CB
:104B06000E9426310E948231E2E2E5BBE0E0EBBB87
:104B1600E7E1E09365001F98F6E1F0936500E09306
:104B26006500EE81E5BBEF81EBBBEFE1FEE1E093D3
:104B36006500F0936500E093650031FF04C0F093D3
:104B46006500E093650026FF10C0F0936500E093D2
:104B5600650031FF06C0F0936500E09365004F5F86
:104B66005F4F220F4F5F5F4FEECF1F9A220F31FF2D
:104B760002C04F5F5F4F4F5F5F4F0C947A25E88509
:104B8600EF5FE8870C947225EC85FD853196EC87FE
:104B9600FD870F5F0C945D251F5F0C9457250E94BF
:104BA6004C3561960895E0E0E0930B03E8EFFFEFE4
:104BB600E0932208F0932308E491EF3F39F0E09167
:104BC6002208F0912308049000920B03A0910B0396
:104BD600A33019F40E94E72102C00E940E1EE3E0F2
:104BE600E0930203E0E0E0930303E1E0E0930103D6
:104BF600E0930003EFEEF0E0E093FF03F093000490
:104C0600EFE3F1E0E0930104F0930204E4E1E093C2
:104C160006030895A0910B03A33069F40E9487311F
:104C26000E9487310E9487310E948731E885EA9386
:104C36000E941B230CC00E9487310E9487310E946C
:104C460087310E948731E885EA930E94711F1DC053
:104C5600A0910B03A33069F40E9487310E9487312B
:104C66000E9487310E948731E885EA930E948B2350
:104C76000CC00E9487310E9487310E9487310E94B2
:104C86008731E885EA930E94D21F29960895A0915C
:104C96000B03A33059F40E948C310E948C31EF81B2
:104CA600EA93EF81EA930E944E250AC00E948C3156
:104CB6000E948C31EF81EA93EF81EA930E943E21B4
:104CC60028960895A0910B03A33029F40E949331EE
:104CD6000E94CC2404C00E9493310E94C0202696D4
:104CE60008950E949A311A930A931BB10CB1E09170
:104CF6009308F0E0EF59F74F0083A0919308AF5F58
:104D0600A0939308A23319F4E0E0E0939308099185
:104D16001991DBC00E949A31E091FA08A091F90836
:104D2600EA1751F0A091FF07A03029F0A0E00A99F8
:104D3600A1E0A03009F401C011C0E091FA08F0E04A
:104D4600EB56F74FE081ECB9A091FA08AF5FA0935C
:104D5600FA08A43619F4E0E0E093FA08B6C0AA937C
:104D6600BA93EA93FA93EFB7EA931A930A931091D8
:104D76009B0000919C00E12FEC7111F00C94282708
:104D8600023021F4E1E0E093930A5FC0E091930AD8
:104D9600E13029F5E0E0E093930A0A3229F00E9417
:104DA600122DE05DE017D1F4E2E0E093930AE0E033
:104DB600E093940A0E94A031E550F74FA2E0A08349
:104DC6000E94A031E0938F0AF093900A0E94A531C9
:104DD600E039A1E0FA0711F40E94A83136C0E230AA
:104DE60071F40093940AE3E0E093930A0E94AF31D2
:104DF600E039A1E0FA0711F40E94A83126C0E33099
:104E060021F50E94AF31E039A1E0FA0711F40E94C2
:104E1600A8310330D1F4E0E0E093930AA091940A1C
:104E2600A63529F4E091FD06E260E093FD06A09127
:104E3600940AA33451F4689423F8E0918F0AF09110
:104E4600900AE093910AF093920A09911991E991D7
:104E5600EFBFF991E991B991A99118951A930E941A
:104E6600B4310E94B931D9F30E94B431E550F74FFD
:104E76001081ADE8BAE00E94742DE039A1E0FA078E
:104E860031F4E0E0F0E0E0938D0AF0938E0AE12F32
:104E9600199108950E949A31E091960BA091950B75
:104EA600EA1781F0E091FC06E03019F0E89421F869
:104EB60008C00E94C0310E94CE3119F4E0E0E093B0
:104EC600960B03C0E89420F821F8E991EFBFF99119
:104ED600E991A9911895E091950BF0E0EB56F54F05
:104EE600A881A083E091950BEF5FE093950B0E945C
:104EF600CE3119F4E0E0E093950B0C94BD2AE0E086
:104F0600E093960BA091950BA13020F00E94C03142
:104F1600689421F80895AA93BA93EA93EFB7EA93AF
:104F2600E0E0E093960B0E94122DEF5FE093FC0603
:104F3600E991EFBFE991B991A99118952A970E9435
:104F4600453520E00E94B4310E94B93121F0A0918C
:104F5600970BA23008F02FC023FE0AC0E091910AF9
:104F6600F091920AE0938D0AF0938E0AE89423F862
:104F760075DF1E2F123029F4E1E0E093970BE0E095
:104F860017C0A091970BA130A9F40E94D3311083CA
:104F9600133039F4E2E0E093970B0E94D331A0E09E
:104FA600A083A091980BAC3328F4E091980BEF5FA7
:104FB600E093980BC7CFA091970BA23011F00C94F9
:104FC600982921E0E091990BE33471F4E0919A0B72
:104FD600E7703E2F303019F40E94421A04C00E9436
:104FE600D9310E94761A9DC1E43471F4E0919A0B8E
:104FF600E7703E2F303019F40E94101D04C00E9445
:10500600D9310E94231D8DC1E73499F5E0919C0B9F
:10501600E73469F4A091FA06A53149F0E0919A0BBC
:10502600E053AE2FE0919B0BE055EA1709F020C044
:10503600E0919A0BE053A8E0B0E00E94B0330E94E2
:10504600EE2C0E94EE2CEFEEF0E00E94F3310E946F
:10505600F82C0E94EE2C0E94EE2C0E941B1AE6EE03
:10506600F3E20E94092D0E94122DF0E00E94C92D44
:1050760058C1E93431F4E0919A0BE370E093FC03F4
:1050860050C1E134E1F4E0919A0BEF70E093020332
:10509600E0919B0BEF70E0930303E0919C0BEF70A4
:1050A600E0930403E0910303A0910203EA1731F4AD
:1050B600A0910303EFE0EA27E093020332C1EC3448
:1050C60039F4E0919A0BE170EA930E94331229C1F8
:1050D600E43511F00C94DD28A0910503A03041F4CD
:1050E600A0919A0BA13320F0A0919A0BAA3308F055
:1050F6001EC0E0919B0BE153A8E9B0E00E94F83195
:10510600E0919A0BE1530E2F0E9402320E948233E5
:105116000E94422F0E94023232960E948233FA93F4
:10512600EA93EAE3F0E00E940B320E941132A0916A
:105136000503A13041F4A0919A0BA13320F0A09170
:105146009A0BA43308F014C0E0919A0BE153AEE435
:10515600B1E20E94F831E0919B0BE153A2E4B1E287
:105166000E941732EAE3F0E00E9422320E941132D6
:10517600A0910503A23041F4A0919A0BA13320F02F
:10518600A0919A0BA43308F014C0E0919A0BE15356
:10519600A8E5B1E20E94F831E0919B0BE153A4E54A
:1051A600B1E20E941732EAE9F0E00E9422320E9440
:1051B6001132B7C0E534A1F4E0919A0BE053E093C5
:1051C6009D06E0919B0BE153E0939E06E0919C0BBC
:1051D600E13311F4E1E001C0E2E0E0932408A1C06C
:1051E600E63459F4A0919A0BA03320F0A0919A0BC3
:1051F600A33308F001C095C002C0E63521F4E0E013
:10520600E0939A0B8EC0E83511F00C948E29E0914C
:105216000503E03031F4E0912408E0930003E1E077
:1052260004C0E1E0E0930003E2E0E093010322FC26
:1052360002C00E943A12689422F8A0919E06E4E108
:10524600EA9FF001A0910103EA9FF001EE5FF0E012
:10525600EA87FB870E94C42EF0E0E887F987E09191
:105266000103A4E1EA9FF001F0E0EE83FF8331E061
:105276000E942732E03011F40C948D29A0919D06EE
:10528600A43120F4A0919E06A33008F041C0E0911D
:105296009D06A3E0EA9FF001EB5DF74FDF01E09189
:1052A6009E06F0E0AE0FBF1F0E942732EC93E091FE
:1052B6009D060E94AE2EDF01E0910003F0E00E9401
:1052C600E832EC87FD87E0910503E03029F0EC85B4
:1052D600FD853A96EC87FD870E942D320E942D327D
:1052E6000E942D32EC85FD850E94F82C0E942D32FD
:1052F600EC85FD850E94C52D0E942732EA93E0E0E9
:10530600EA930E94BC19E0919D06EF5FE0939D062B
:105316003F5FAECF06C0E93521F40E94D716E89468
:1053260022F8E0E0E093970BE22F0E944C3560965E
:105336000895A0E020FCA1E0A03029F4E091FD064C
:10534600E270E23009F010C00E943232E05DEA936A
:10535600C2DDE6E5EA93BFDDE2E30E943A32ED7F85
:10536600E093FD06689420F8A0E020FCA1E0A030C0
:1053760029F4E091FD06E370E13009F020C00E94B7
:105386003232E05DEA93A7DDE4E5EA93A4DDE0913D
:10539600FA06EA93A0DDE0911E08E295EF70EA9323
:1053A60026D0EA9398DDE0911E08EF70EA931FD0AD
:1053B6000E943A32EE7FE093FD06689420F8A0E062
:1053C60020FCA1E0A13049F4A0E021FCA1E0A0303E
:1053D60021F4A091FC06A03009F001C090DDE09117
:1053E600FC06E03019F0E150E093FC060895A88130
:1053F600AA3020F4E881E05D0C94BD2AA881AA3089
:1054060020F0E881E95C0C94BD2AE8E50C94BD2AFD
:105416000E9444320E9449320E94F3310E944C326B
:105426000E9444320E949F2DE4E1F0E00E94F33195
:105436000E944C32E2EDF0E0FA93EA930E94493280
:105446000E94F3310E944C32E2EDF0E0FA93EA93C7
:105456000E949F2DE4E1F0E00E94F3310E944C325D
:10546600E4E1F0E0FA93EA930E944432E8ECF0E0DB
:10547600FA93EA93ECE3F0E00E9452320E9449323A
:105486000E94F3310E945832E2EDF0E00E94F331BF
:105496000E94F3310E945832EFE0E0930303E2E00A
:1054A600E0930003E0930103E5E5F0E0FA93EA9365
:1054B600EEE1F0E00E94C52DECEEF3E20E94092D2C
:1054C6000E94FE2CE0E0E09303030895EEE5F1E28E
:1054D600FA93EA93EAEBEA93EAEFF0E0FA93EA93B7
:1054E600E4E0EA93E6E2EA93EEE0EA930E944A26D3
:1054F600E6EFF1E2FA93EA93EAEAEA93E7E0F1E00B
:10550600FA93EA93E8E0EA93E2E3EA93E1E0EA93C6
:105516000E944A260895E991F991A991B991CD0180
:1055260061916D936623E1F7FC010895E991F99184
:10553600A991B991CD0105900D920020E1F7FC01EA
:105546000895A991B991EE27FF276D91662311F071
:105556003196FBCF0895AA27BB27E991F9910590CB
:10556600002011F01196FBCFFD0108955D9BFECF43
:10557600E881ECB9219608951A930A93AC81BD810E
:105586000E9478333097C1F0AA81BB810E9478339C
:105596008F01309749F00230E0E01E0760F0F80115
:1055A60031978F01ED93FC93AC81BD810E94742DE0
:1055B6003197AE81A08303C0EE81EA93D7DF1981CC
:1055C6000881279608952C970E94453510E0E88DAE
:1055D600F98D3196E88FF98F3197E4912E2FE030CF
:1055E60011F40C94A22CE12FE03039F4253211F499
:1055F60011E002C00E945D32A1C1E130C1F4253242
:1056060019F40E945D3299C112E0E0E0E98B00E0F6
:105616002D3211F401E092C12B3219F4EBE2E98B41
:105626008DC1203219F4E0E2E98B88C102C0E23074
:1056360039F450E013E0203311F400687FC102C052
:10564600E330A1F4203310F02A3308F009C0A52F67
:10565600EAE0EA9FF0015E2FE22FE0535E0F6EC193
:1056660040E02E3211F414E069C110C0E430A1F418
:10567600203310F02A3308F009C0A42FEAE0EA9F8D
:10568600F0014E2FE22FE0534E0F58C12C3619F47D
:10569600026015E053C104C0E53011F00C94A12C52
:1056A600E22FE33649F40E946832EE89FF89A4812D
:1056B600AA930E946E3241C1E33741F40E946832D8
:1056C6000E9478320E94A42A1E2F0AC0E037A1F455
:1056D6000E9468320E9478320E94AE2A1E2F08600D
:1056E6000F77403011F0411708F001C0142F40E049
:1056F600E0E0E88B30E078C0E43611F0E93611F4EA
:10570600046002C0E537A1F4EAE0E88B01FF08C0B7
:10571600E0E0FAEC6AE97BE30E94862D1AE023C0FA
:10572600E0E1F7E260E070E00E94862D15E01BC024
:10573600E83511F4086004C0E83711F00C94A02C89
:10574600E0E1E88B01FF08C0E0E0F0E060E070E136
:105756000E94862D18E007C0E0E0F0E160E070E00E
:105766000E94862D14E0403011F00F7701C041E011
:1057760001FF08C00E946832AE89BF8914960E9454
:105786007C3315C002FF0AC00E946832AE89BF8909
:1057960014960E9478330E94B53209C00E9468327E
:1057A600AE89BF8914960E94783366277727EC87DF
:1057B600FD876E877F8702FF16C0AF85AA2362F436
:1057C600EC85FD856E857F850E949F32EC87FD877F
:1057D6006E877F87EDE2E98BE989E03019F01F5F7C
:1057E6004F5F01C00B7F342F00FD14C0151710F456
:1057F600351708F00FC007FF08C002FF04C00B7F73
:105806002989115001C020E301C020E20E945D32C7
:105816005150ECCF1417B0F4006102FF0AC00B7FA1
:10582600E989EA930E946E32503009F051501150C6
:105836004150E0E3EA930E946E32503009F0515035
:105846004150E8CF312FE889E030D1F43030B9F05B
:1058560003FF08C0EE81FF813196EE83FF83319707
:10586600E49105C0AE81BF81ED91AE83BF83EA931B
:105876000E946E32503009F051503150E7CF53C07C
:105886000E9482320E9418332E2F2A3030F003FFF6
:1058960002C0295C01C0295A01C0205D04FD23C055
:1058A600213350F40E948B2DA130E0E0BE07E0E0EA
:1058B6008E07E0E09E0709F40BC0431740F4531728
:1058C60010F000FF01C014C020E207FF0CC020E367
:1058D600006102FF08C00B7FE989EA930E946E32DD
:1058E600503009F051500E945D32503009F051504D
:1058F60031500E9482320E945333EC87FD876E87B7
:105906007F87E8890E948B2DFF27662777270E94CD
:1059160018330E94862DE885F9856A857B850E9465
:105926003D3509F0ADCF00FF08C0503031F0515081
:10593600E0E2EA930E946E32F8CF10E048CE0E9471
:105946004C356A960895FF92F82E22971A930A9379
:10595600DE010E9497328D01DE0116960E94973273
:105966000E947833EA83FB83DE0114960E94973205
:105976000E947833FA93EA931A930A930E94792E37
:105986000E94EE2C20DEAA81BB81E0E0EC93198117
:1059960008812496FF900895A991B991EE270024D5
:1059A60060E8E894162E169407941E2A1EF0A01599
:1059B600B10518F0A019B109E62BB7FBAA0FBB1F5A
:1059C600669580F70895E991F99130971AF4E09574
:1059D600F09531960895E0E0F0E0FA93EA930895A1
:1059E600E091FF03F09100040895FA93EA93EFE043
:1059F600EA930C940D26E1E0E0930003E0930103A3
:105A06000895E6E0F0E0FA93EA930895FA93EA93AC
:105A16000C941417E7E0F0E0FA93EA930895A8E0EF
:105A2600B0E00E949C330895E0918D06F0918E06B9
:105A36000895E0918906F0918A060895EAE0E093D8
:105A46006100E5E0E09362000895EA930E946D121A
:105A5600E0939B06F0939C060895E093620088EC21
:105A660090E00197F1F70895E093610088EC90E0EB
:105A76000197F1F70895AE0FBF1FE3E0F0E00E9433
:105A860013330895FA93EA931A930A930C947812AF
:105A9600FA93EA933A932A930C947812A09191067A
:105AA600B09192060895A0919306B0919406089538
:105AB600A5E8B6E0ED91FD913196FE93EE9308953B
:105AC600A0918506B09186060895E0937906F09335
:105AD6007A060895E0E0F0E0E0938506F093860606
:105AE6000895ED91FD913196FE93EE930895A0E011
:105AF600B0E00E94983308950E949133EA1BFB0B95
:105B06000E94B5320895E887F9876A877B870895EA
:105B1600A885B9858A859B850895A2E0B0E00E9494
:105B260098330895A4E0B0E00E9498330895A6E063
:105B3600B0E00E9498330895E2E3F0E0FA93EA9326
:105B46000895FA93EA930C948B32A0918106B09152
:105B560082060895E0EAF0E0FA93EA930895EA935C
:105B66000E94131AE1E0E09300030895EAE0EA9345
:105B76000E94A416E0919106F091920608950E9463
:105B8600A833DACFFA93EA930C94361AFA93EA9387
:105B96000C94F416E8E1F0E0FA93EA93E8E2F0E018
:105BA60024CFE7EDF0E0FA93EA93D4CFE2E0E09376
:105BB6000003E9E6F0E0FA93EA930895EAE0EA934F
:105BC6000E94A416E0919306F091940608950A9215
:105BD6001A92FA926A937A938A939A93AA93BA93A9
:105BE600EA93FA93EFB7EA930895ACE01A9FF001AF
:105BF600E45FFC4FE0810895ACE01A9FF001EB5E94
:105C0600FC4F08951A93E1E0EA930C94A31AEAE094
:105C1600F0E097CFE093E006F093E1060895A981BE
:105C2600BA81EE27A10FBE1FEC910895FE01FA93EB
:105C3600EA9308950E94863384E00E94A62C289653
:105C4600F5CFF801AA81BB81EA0FFB1FE491089505
:105C5600E091E306A6EEB6E0F0E0EE0FFF1F089532
:105C6600E091E206A6EEB6E0F0E0EE0FFF1FEA0FC7
:105C7600FB1F0895E981ACE0EA9FF0010895EF73F8
:105C8600A9E2EA9FF001E757FB4F0895EF73ABE0F7
:105C9600EA9FF001EB5FFB4F0895ACE01A9FF0011D
:105CA600E15FFC4F0895ACE01A9FF001E35FFC4F03
:105CB600DF010E9478330895ACE01A9FF001E35F9C
:105CC600FC4F608171811A9FF001EF5EFC4FE0810D
:105CD600DB01F0E00895A083ACE01A9FF00108957F
:105CE600ACE01A9FF001EA5EFC4F0895FE0136967D
:105CF600FA93EA930895FA93EA930C948E2AA9E20A
:105D06000A9FF001E757FB4FE081E0300895A9E2D2
:105D16000A9FF001E757FB4FFA93EA93FE01389684
:105D2600EACFABE00A9FF001EB5FFB4FE081E0308A
:105D36000895E091E006F091E1060895A0EEB6E040
:105D4600ED91FD913296FE93EE930895E081F0E099
:105D5600E60FF71F0895F0E0ACE0B0E00E94E832ED
:105D660008951A930A933A932A930895E0910103AA
:105D7600F0E00895FA93EA93ED81EA93ED81EA93D0
:105D86000895E0910003ACE0EA9FF0010895F0E089
:105D9600EA0FFB1F0895E0930703F09308030895A5
:105DA6001A93E1E0E0930103E093000310E0089505
:105DB600DF010E947833DF01EB81FC810895DF016A
:105DC6000E947833DF01E981FA810895EF81F88531
:105DD600EA1BFB0B0895FE01EB5BFF4FE081ACE095
:105DE600EA9FF001EA5EFC4FE0810895FE01EB5B5D
:105DF600FF4FE081ACE0EA9FF0010895ECE8F0E0A7
:105E06000E9482330895DE01A05CBF4FED93FC93A0
:105E16000895FE01E85BFF4F0190F081E02D0895A3
:105E2600FA01E00FF11FFA93EA930895E0E0EA938E
:105E36000C942B261A930A93FE01EC5BFF4F0190FC
:105E4600F081E02DE20FF31F0895FA93EA93E8CF6D
:105E5600E0DFE20FF31FFA93EA93E8CFE0E0EA937C
:105E66000C940D26FA93EA933A932A930895E5E063
:105E7600F0E0FA93EA93CDDFFA93EA93EFCFFA9341
:105E8600EA935A934A930895DE01AC5BBF4FAC91F7
:105E96000895DA01F0E00895DF01FE01EE5BFF4FA1
:105EA6000190F081E02DAE17BF070895FE01EE5B6D
:105EB600FF4F0190F081E02D0895E2E0F0E00E94AE
:105EC60013330895A0DFDE01AF5BBF4FAC91AA2369
:105ED6000895ECE0EA9FF001A0910003EA9FF0012B
:105EE6000895AE1BBF0BE9CFECADF0E0E00FF11F5C
:105EF60008953196FA93EA93D9DFE20FF31F3196AC
:105F060041CEFA93EA93D2DFE20FF31F3BCEEFAD19
:105F1600F0E0DE011696AE0FBF1FEC910895EA93EE
:105F2600EBADEA930E94BC19EFADEF5FEFAF0895BA
:105F3600F0E0DE011696AE0FBF1FAC9108950E94E9
:105F4600E832E20FF31FDF01B1DFEE0FFF1FEA0FAA
:105F5600FB1F08950E94E8320E94B5320E94273442
:105F66000895E98DFA8DE21BF30BFA93EA930895EF
:105F7600FA93EA93F901AD8DBE8DEA0FFB1FFA93F2
:105F8600EA930895FA93EA93EA8DEA930C942B2602
:105F9600EBE1E0936500E4E6F0E0D3CDFA93EA9313
:105FA6000C94EA1DEA93E1E0F0E0F8CFE3E0EA932F
:105FB600E0E3F0E1F3CFE4E0EA930DCDEA93E7E026
:105FC600F7E0ECCF0E94EA1DE1E5EA93EFEEF0E0A0
:105FD600E5CF0E94EA1DE3E5EA93EFE3F1E0DECFC9
:105FE6000E944535EE81AEEDB0E2F0E0EE0FFF1F08
:105FF600EA0FFB1F0E9482338F010895E985FA8517
:10600600AD85BE850895AD85BE85EFEEF0E0EA1B51
:10601600FB0BE987FA870895EF81F885AB85BC8588
:106026000895AB85BC85EFE3F1E0EA1BFB0BEF833C
:10603600F8870895EA93EE85FF85B0CFEA93EA855F
:10604600FB85AE85BF850895EA0FFB1FA7CFEA93B0
:10605600EC85FD85A3CFEA93E885F985AC85BD85FA
:106066000895EF81F885E017F1070895EB85FC8523
:10607600AF81B885AE17BF0708950D851E85ED85DE
:10608600FE85E987FA870D871E870B851C85EB85BC
:10609600FC85EF83F8870B871C870895ED85FE85C1
:1060A600A985BA85AE17BF070895AD85BE85E98572
:1060B600FA85EA1BFB0B0895FA93EA930C94E62CF7
:1060C600AB85BC8583CEAF81B885EB85FC85EA1BA5
:1060D600FB0B0895D9010E94E8320F010895D00103
:1060E6000E941333AF01E0E2EA93FA01AE85BF8561
:1060F600ABCFE2E2EA931A930A930C94EA1DEA9371
:10610600F901AC85BD850895A985BA85ED85FE851D
:10611600EA1BFB0B0895D0010E941333AF01E0E2A6
:10612600EA930895E1E2EA93FA01AC85BD858CCF46
:10613600AEEDB0E2F0E0EE0FFF1FEA0FFB1F0E948C
:106146008233EE83FF830895EC85F0E0EE0FFF1FA8
:106156000E94A732E887F9873091000310E008957E
:10616600EA85F0E00E94A932DF01E32FF0E00E9409
:10617600E832AF85B889EA0FFB1FAF01EA85A8852B
:10618600B98505CEE0E2EA935A934A930C94EA1D48
:10619600E885F0E00E94A932DF01E32FF0E00E94DB
:1061A600E832AE85B0E0EA0FFB1FAF01EF85F88954
:1061B60024913196EF87F88B0895FA93EA930C941D
:1061C600BA21EA93E4E0F0E0F8CFE6E1EA93E8ECFE
:1061D600F0E0F3CFEA93E2E0F0E0EFCFEA93E1E01C
:1061E600F0E0EBCFE8E2F0E0ACCC0E944535EE8182
:1061F600AEEFB0E2F0E0EE0FFF1FEA0FFB1F0E94CA
:1062060082338F010895E2E0EA93EE85FF850E94CE
:10621600B032D3CFAE0FBF1FFD010E94B032CDCF3B
:10622600E6E0EA93EC85FD850E94B032C6CF0E9477
:10623600BA21E5E0EA93EFEEF0E0BFCFE9E0EA93BA
:10624600EFE3F1E0BACF0E94B032B7CFEA93EC8524
:10625600FD85F070B2CFE6E0EA93EE85FF85F3CFD9
:10626600E7E0EA93EE85FF85F070A7CFD0010E94A4
:106276001333AF01E2E0EA93FA01AE85BF85CACFD8
:10628600E3E0EA93FA01AE85BF85AE0FBF1FEFEFDD
:10629600F0E0EA23FB2391CFA21BB30BEFEFF0E074
:1062A600EA23FB238ACFE2E2EA931A930A930C9439
:1062B600BA21AE0FBF1FEFEFF0E0EA23FB237DCF3D
:1062C600D0010E941333AF01E2E0EA930895E6E0BD
:1062D600EA93FA01AC85BD859DCFE7E0EA93FA0122
:1062E600AC85BD85E6CFAEEFB0E2F0E0EE0FFF1F66
:1062F600EA0FFB1F0E948233EE83FF830895E3E0DB
:10630600EA93FA01F07059CFEF81F885FA93EA9390
:106316000895EE81FF81FA93EA93EF81EA93089557
:10632600EC81FD81FA93EA93EC81FD8123CDAA935A
:10633600EA93FA93EFB7EA930895E0918B0AF09106
:106346008C0A0895ABE8BAE0CCCBE0E0F0E0E0934D
:106356008B0AF0938C0A0895F0DFE550F74F00831F
:10636600F1CFE0918D0AF0918E0A0895A0918B0AE3
:10637600B0918C0AEA17FB070895E091960BF0E0BE
:10638600EB56F54FE081E0939C00E091960BEF5FB2
:10639600E093960B0895F0E0E030A1E0FA07089547
:1063A600E091980BF0E0E756F44F0895E32FE150A3
:1063B600A8E9B0E0F0E0EE0FFF1FEA0FFB1F0E9416
:1063C6008233FA93EA93E32FA8E9B0E0F0E0EE0F08
:1063D600FF1FEA0FFB1F0E948233FA93EA93089588
:1063E600FA93EA93E4E1F0E00895F0E0EE0FFF1F80
:1063F600EA0FFB1F0E9482333396AF010895E02F08
:10640600AEE1B1E2F0E00E94AB32EA0FFB1F089565
:10641600FA93EA93E0919C0BEA93DDCAEDE9FBE07F
:10642600FA93EA930C948517F0E0EE0FFF1FEA0F3C
:10643600FB1F0E9482333396EE87FF8720CDFA93A7
:10644600EA93EAE4F0E0E4CFE32FF0E0E756F44F16
:10645600E0810895EC85FD85FA93EA930895E0E0DE
:10646600E093950BE2E0EA930E946E27D8CAEA937E
:106476000E946E27E3E0EA930E946E27E091FD06F4
:106486000895EAE0F0E0FA93EA930895EAE0F0E08E
:10649600A7CFFA93EA93ECE0EA930C945D1DFA9386
:1064A600EA93ECE0EA930C940D26FA93EA93E8E279
:1064B600F0E0F5CF2A93ED89FE89FA93EA93FE017F
:1064C6007596FA93EA930C94BF2AEE89FF8934975E
:1064D600EE8BFF8B0895ED89FE89FA93EA93FE0110
:1064E6007596FA93EA930C94BF2AAE89BF891496DF
:1064F6000E947833EE83FF83FA93EA930895E88542
:10650600F9856A857B85AC85BD858E859F850895D1
:10651600E991F991309639F080EA9FE00197F1F719
:10652600A8953197C9F708950024AF0DB01D0895B9
:10653600F195E195F0400895F09560957095E19597
:10654600FF4F6F4F7F4F0895EE0FFF1FEE0FFF1F98
:10655600EE0FFF1FEE0FFF1F0895EF2FFF27E7FD3A
:10656600FFEF08956F2F660F660B762F0895EA17D3
:10657600FB07E1E00CF0EE270895FA9FF02DEB9F64
:10658600F00DEA9FE02DF10D08957A9F702D6B9F17
:10659600700DF89F700DE99F700D6A9F602D710D4B
:1065A600FB9F600D711DE89F600D711D8827FA9F86
:1065B600F02D610D781FEB9FF00D611D781FEA9F8E
:1065C600E02DF10D681F781F08956ED0D6DF0EF40A
:1065D600AFDF089577D0D9DF0EF4AEDF089500243B
:1065E60098E0AA0F001C0E1A10F40E0E01C0A1604E
:1065F6009A95B9F7EA2FA02D08950024112490E169
:10660600AA0FBB1F001C111C0E1A1F0A18F40E0E2F
:106616001F1E01C0A1609A9599F7FD01D00108954A
:1066260043D0EBDF0EF484DF08953F934F935F93DF
:10663600002411244427552730E2AA0FBB1F881FC8
:10664600991F001C111C441F551F0E1A1F0A460BCA
:10665600570B28F40E0E1F1E461F571F01C0A160C0
:106666003A9559F7FD01BC01D001CA015F914F91DE
:106676003F91089527D0D9DF0EF45EDF0895AFDF8E
:10668600EA2F0895E894B7FF04C0A095B095119637
:106696006894F7FD4DDFB1DFFD010EF449DF089583
:1066A600C4DFFD01BC010895E894F7FF02C040DF96
:1066B6006894B7FF06C0A095B095119600F80394AC
:1066C60000FA0895E89477FF02C036DF689497FFD2
:1066D6000BC00024A095B095809590951196801DCD
:1066E600901D00F8039400FA0895ED91FC9111971E
:1066F6000895ED91FD916D917C9113970895059004
:10670600F491E02D08957A936A93FA93EA930895A3
:10671600182E862F612D192E972F712D1B2EBF2F08
:10672600F12D1A2EAE2FE12D0895119602D0FE2FCF
:106736001197E199FECFFF93FFB7F894AEBBBFBBAD
:10674600E09AEDB3FFBFFF91089507D01196EF933E
:10675600EF2F03D0EF9111970895E19B02C0A89502
:10676600FCCF9FB7F894AEBBBFBBE09A8DB3E817DA
:1067760019F0EDBBE29AE19A9FBF0895552342F4C2
:10678600503811F4E0FF04C03196691F791F6BF091
:1067960050E8572711F45F93C8C05F3F31F0660F8A
:1067A600000C57956795752F08955F9300200AF0A2
:1067B600C8C0C1C050E8192E1522880F991F952709
:1067C600550F879550E8072E0522660F771F752708
:1067D600550F67950895689401C0E8945F93F2DFBA
:1067E600703818F07F3F08F4A0C056E1571BAAF492
:1067F600519558300EF4593030F0EFEFFFEF6FEF50
:106806007FE777F91AC077275523B9F0EE0FFF1FF8
:10681600661F771F5A95D1F710C07727583028F092
:10682600EF2FF62F672F5850F9CF552331F0769575
:106836006795F795E7955A95D1F700200AF47CDE1F
:106846005F910895689401C0E89430976040704065
:10685600B1F0002426F0772312F400946DDE172E93
:106866007EE1112032F07A95EE0FFF1F661F111C94
:10687600F9CFEF2FF62F612D5F938ADF5F91089591
:106886004F93AF01FD01DA01AB01BC01CA01402DF6
:10689600012C142E4F910895EA0FFB1F681F0895CF
:1068A600E095F0956095EF5FFF4F6F4F08955F930A
:1068B60081DF903849F150E81526703821F1572FBD
:1068C600591B13F112F4DCDFFACF583118F0AA275E
:1068D600BB278827583028F0AB2FB82F8827585069
:1068E600F9CF552329F08695B795A7955A95D9F7E7
:1068F600502D512562F0D0DF38F46795F795E7956E
:10690600739513F41EC0BCDF43DF5F910895EA1B45
:10691600FB0B680B51F010F40094C2DF6623A2F360
:10692600EE0FFF1F661F7A95CBF7EE27FF27662728
:1069360077275F910895EFEFFFEF6FE77FEF5F91A6
:106946000895EFEFFFEF6FE77FE75F9108955F939D
:1069560031DF703851F3903841F301240894791FE0
:1069660023F41CF300203AF3ECCF0F921F932F93DE
:106976003F934F93112722279927689FA0018F9F46
:10698600302D410D591F6B9F300D411D591F8E9F94
:1069960027D0BF9F25D06A9F23D0BE9F1DD0AF9F13
:1069A6001BD0AE9F110D291F391F491F591FE32FF9
:1069B600F42F652F522F4F913F912F911F910F90DA
:1069C60066232AF0550FEE1FFF1F661F02C0739540
:1069D6004BF2D4DE5F910895100D211D391F02C0C0
:1069E600200D311D491F591F08955F93E3DE70384E
:1069F60021F411200AF49FCFA4CF903809F495CF43
:106A060001240894970B1BF4D4F30020F3CF792FBD
:106A16001F932F933F934F93112411272227332738
:106A26004427552790E2AE17BF078607410730F087
:106A3600AE1BBF0B860B410B089401C08894551FF3
:106A4600221F331F111CAA1FBB1F881F441F9A95A4
:106A560051F7F901612D4F913F912F911F916623B7
:106A660032F0550FEE1FFF1F661F7A9543F286DE42
:106A76005F910895309760407040089500240A168B
:106A86000B0608955A934A933A932A931A930A93B4
:106A960008955D814C813B812A8119810881089581
:00000001FF
